:020000040000FA
:1000000094EF37F0F76A140FF66E000EF72209002E
:10001000F5501200000000000000005F0000000723
:10002000000700147F147F14242A7F2A1223130848
:10003000646236495522500005030000001C22412D
:10004000000041221C0014083E081408083E08085D
:100050000050300000080808080800606000002018
:10006000100804023E5149453E00427F4000426173
:100070005149462141454B311814127F10274545FF
:1000800045393C4A49493001710905033649494916
:1000900036064949291E0036360000005636000053
:1000A00008142241001414141414004122140802EC
:1000B00001510906324979413E7E1111117E7F4975
:1000C0004949363E414141227F4141221C7F4949F5
:1000D00049417F090909013E4149497A7F080808D9
:1000E0007F00417F41002040413F017F08142241B1
:1000F0007F404040407F020C027F7F0408107F3E1B
:100100004141413EF76A140FF66E010EF7220900D5
:10011000F55012007F090909063E4151215E7F0911
:10012000192946464949493101017F01013F4040B3
:10013000403F1F2040201F3F4038403F63140814B9
:100140006307087008076151494543007F4141003A
:1001500002040810200041417F0004020102044013
:1001600040404040000102040020545454787F482D
:100170004444383844444420384444487F38545434
:100180005418087E0901020C5252523E7F080404A2
:100190007800447D40002040443D007F102844000A
:1001A00000417F40007C041804787C0804047838FF
:1001B000444444387C14141408081414187C7C0833
:1001C0000404084854545420043F4440203C404018
:1001D000207C1C2040201C3C4030403C44281028FF
:1001E000440C5050503C4464544C44000836410088
:1001F00000007F0000004136080010080810087851
:1002000046414678F76A140FF66E020EF72209008F
:10021000F55012004272696768746E65737300006E
:10022000F76A300FF66E020EF7220900F550120041
:1002300041646A7573740000F76A480FF66E020E27
:10024000F7220900F550120054656368446573692C
:10025000676E2E626500F76A660FF66E020EF72271
:100260000900F5501200566F703D202575200000E2
:10027000F76A800FF66E020EF7220900F5501200A1
:1002800020202020202020202020202020200000AE
:10029000F76AA00FF66E020EF7220900F550120061
:1002A00020636172643F2000F76AB80FF66E020E99
:1002B000F7220900F550120043617264203F2020AC
:1002C000202020202000F76AD60FF66E020EF722BB
:1002D0000900F550120061636D64383D25782000F7
:1002E000F76AF00FF66E020EF7220900F5501200C1
:1002F0004361726420426F6F742E2E2E0000F76AE5
:100300000E0FF66E030EF7220900F55012007374FB
:100310006174313D20254C782000F76A2A0FF66E73
:10032000030EF7220900F550120073746174323D18
:1003300020254C782000F76A460FF66E030EF72250
:100340000900F5501200534448433D202578200011
:10035000F76A600FF66E030EF7220900F5501200DF
:100360002020534420426F6F742E2E2E0000F76A17
:100370007E0FF66E030EF7220900F550120053446B
:10038000484320426F6F742E2E2E0000F76A9C0F98
:10039000F66E030EF7220900F550120073746174B3
:1003A000333D20254C782000F76AB80FF66E030E17
:1003B000F7220900F550120061636D6434313D206D
:1003C00025782000F76AD40FF66E030EF722090095
:1003D000F55012004D4D43204D4F44452000F76A23
:1003E000EE0FF66E030EF7220900F5501200204DB5
:1003F0004D4320426F6F7400F76A080FF66E040ECB
:10040000F7220900F550120053656356423D256CF2
:1004100078200A0D0000F76A260FF66E040EF72208
:100420000900F550120042705365633D20256C7839
:10043000200A0D00F76A440FF66E040EF722090039
:10044000F550120053656370436C753D202578208C
:100450000A0D0000F76A640FF66E040EF722090019
:10046000F5501200525365633D20254C78200A0D4B
:100470000000F76A820FF66E040EF7220900F550AD
:1004800012004661744E3D202578200A0D00F76A5F
:100490009E0FF66E040EF7220900F5501200536508
:1004A00063466174313D20254C78200A0D00F76ABF
:1004B000BE0FF66E040EF7220900F55012004641F9
:1004C00054315F6C62615F73746172743D20254CBE
:1004D00078200A0D0000F76AE60FF66E040EF72288
:1004E0000900F550120053704661743D20254C7888
:1004F000200A0D00F76A040FF66E050EF7220900B8
:10050000F550120052446972456E744E3D20254CE0
:1005100078200A0D0000F76A260FF66E050EF72206
:100520000900F5501200536563526F6F744469728D
:100530003D256C78200A0D00F76A480FF66E050E0F
:10054000F7220900F5501200456E64536563526F3F
:100550006F744469723D256C78200A0D0000F76ABB
:100560006E0FF66E050EF7220900F5501200536566
:10057000637046415433323D256C78200A0D0000EB
:10058000F76A900FF66E050EF7220900F55012007B
:10059000436C75526F6F744469725F4641543332D5
:1005A0003D256C78200A0D00F76AB80FF66E050E2F
:1005B000F7220900F55012006C6261526F6F7444AB
:1005C00069723D256C78200A0D00F76ADA0FF66E25
:1005D000050EF7220900F550120021212042705328
:1005E0006563206973206E6F7420353132202121BC
:1005F000200A0D00F76A040FF66E060EF7220900B6
:10060000F55012005363616E6E696E672E2E2E00D8
:10061000F76A200FF66E060EF7220900F550120059
:100620002A2A7365637363616E3D256C7520000033
:10063000F76A400FF66E060EF7220900F550120019
:10064000726F777363616E3D256C75200000F76AE9
:100650005E0FF66E060EF7220900F5501200726F5B
:10066000777363616E313D256C752000F76A7C0FEE
:10067000F66E060EF7220900F5501200726F7773BE
:1006800063616E323D256C750A0D0000F76A9C0FA0
:10069000F66E060EF7220900F550120044454C2074
:1006A0000000F76AB20FF66E060EF7220900F55049
:1006B00012004C464E200000F76AC80FF66E060E78
:1006C000F7220900F5501200454E44312000F76A28
:1006D000DE0FF66E060EF7220900F5501200454EA9
:1006E00044322000F76AF40FF66E060EF722090076
:1006F000F55012000000F76A060FF66E070EF7229B
:100700000900F55012002028726F6F74292025759A
:100710000000F76A220FF66E070EF7220900F55067
:1007200012002A2A2A46494C453D2000F76A3C0F10
:10073000F66E070EF7220900F55012006469725F29
:100740006E756D6265723D2575200000F76A5C0F5D
:10075000F66E070EF7220900F55012006E657874E8
:10076000436C75737465723D25386C75200A0D00F5
:10077000F76A800FF66E070EF7220900F550120097
:100780006363323D256C75200A0D0000F76A9C0FEB
:10079000F66E070EF7220900F55012005449543244
:1007A0000000F76AB20FF66E070EF7220900F55047
:1007B0001200545045310000F76AC80FF66E070E5C
:1007C000F7220900F550120054434F4E0000F76A1B
:1007D000DE0FF66E070EF7220900F5501200545294
:1007E000434B0000F76AF40FF66E070EF72209007C
:1007F000F550120054414C420000F76A0A0FF66EA1
:10080000080EF7220900F550120054454E4300002F
:10081000F76A200FF66E080EF7220900F550120055
:10082000545945520000F76A360FF66E080EF7224B
:100830000900F5501200434F4D4D0000F76A4C0F70
:10084000F66E080EF7220900F55012002020202035
:100850002020202020202020202020202020202098
:1008600020202020202020200000F76A7A0FF66E3A
:10087000080EF7220900F5501200202A2A2A202506
:1008800073202A200000F76A960FF66E080EF722F2
:100890000900F55012002573202A2A2A2000F76A41
:1008A000AE0FF66E080EF7220900F55012006B62CB
:1008B00070733D202575200A0D00F76ACA0FF66E89
:1008C000080EF7220900F55012006B6270735F6426
:1008D00065633D20256C75200A0D0000F76AEC0F5A
:1008E000F66E080EF7220900F550120020736563BA
:1008F000735F746F743D256C75200000F76A0C0FF0
:10090000F66E090EF7220900F55012007461675F58
:1009100073697A653D20256C75200A0D0000F76A21
:100920002E0FF66E090EF7220900F55012002D2049
:10093000536F6E67205469746C65202D0000F76A50
:100940004E0FF66E090EF7220900F55012002D2DFC
:10095000202041727469737420202D2D0000F76AE5
:100960006E0FF66E090EF7220900F5501200202DC9
:100970002D2D2000F76A840FF66E090EF72209006C
:10098000F5501200205642522000F76A9A0FF66E78
:10099000090EF7220900F55012000A0D30323020FE
:1009A0002D204563686F4D7033204D4D432F5344C8
:1009B000206D703320506C61796572200A0D0A0D2C
:1009C0000000F76AD20FF66E090EF7220900F55003
:1009D0001200204563686F4D70332076312E34202D
:1009E0000000F76AF20FF66E090EF7220900F550C3
:1009F00012004D4D432F5344204361726400F76A47
:100A00000E0FF66E0A0EF7220900F5501200202094
:100A10004D703320506C6179657220200000F76AB8
:100A20002E0FF66E0A0EF7220900F55012004469E7
:100A300061677300F76A440FF66E0A0EF722090029
:100A4000F550120053687566666C6500F76A5C0FB6
:100A5000F66E0A0EF7220900F55012004D4D432F95
:100A6000534420696E697420646F6E65200A0D001E
:100A7000F76A800FF66E0A0EF7220900F550120091
:100A80004D4D432F5344207265616420626F6F7433
:100A900020646F6E650A0D200000F76AAA0FF66EDB
:100AA0000A0EF7220900F5501200767320696E696C
:100AB0007420646F6E650A0D2000F76ACA0FF66E27
:100AC0000A0EF7220900F5501200546F74616C2071
:100AD000536F6E67733D20254C75200A0D00F76A31
:100AE000EE0FF66E0A0EF7220900F5501200646947
:100AF000725F6E756D6265722025753D2000F76A24
:100B00000E0FF66E0B0EF7220900F5501200746FEF
:100B100074616C646972733D202575200A0D0000B4
:100B2000F76A300FF66E0B0EF7220900F55012002F
:100B300063757272656E74736F6E673D25334C75A5
:100B40002F254C752000F76A560FF66E0B0EF72214
:100B50000900F55012006C62615F73746172743D3C
:100B6000256C75200000F76A760FF66E0B0EF722E3
:100B70000900F5501200736F6E675F6C62615F6C05
:100B8000656E6774683D256C75200A0D0000F76A74
:100B90009E0FF66E0B0EF7220900F55012007374CB
:100BA00061727420706C6179696E672E2E0A0D0077
:100BB000F76AC00FF66E0B0EF7220900F55012000F
:100BC000204469726563746F726965732020000048
:100BD000F76AE00FF66E0B0EF7220900F5501200CF
:100BE0002A2A2A2A2A2A2063757272656E74646919
:100BF000723D202575200A0D0000F2CF5AF3F29EB7
:100C0000010EA96EA69CA69EA680A85003015ABFFD
:100C1000F28E010B016E0101409501B04085F2CFCB
:100C20005AF3F29E020EA96EA69CA69EA680A8501C
:100C300003015ABFF28E010B016E0101409701B012
:100C4000408780AA2FD040A517D0010EA96EA86AB0
:100C5000A69CA69EA684F2CF00F0F29E0F01550E30
:100C6000A76EAA0EA76EA682A6B2FED7A6940050C3
:100C7000F2120101409516D0010EA96EA86EA69C35
:100C8000A69EA684F2CF00F0F29E0F01550EA76E2D
:100C9000AA0EA76EA682A6B2FED7A6940050F212A4
:100CA0000101408584A030D040A717D0020EA96E64
:100CB000A86AA69CA69EA684F2CF00F0F29E0F0121
:100CC000550EA76EAA0EA76EA682A6B2FED7A69450
:100CD0000050F2120101409717D0020EA96E010ECA
:100CE000A86EA69CA69EA684F2CF00F0F29E0F01ED
:100CF000550EA76EAA0EA76EA682A6B2FED7A69420
:100D00000050F21201014087000138EF39F0F2CFB4
:100D10005AF3F29EA96AA69CA69EA680A85003013B
:100D20005ABFF28E02012D6F2D517F0816E3A00EDF
:100D30002D6FA96AA86EA69CA69EA684F2CF00F08D
:100D4000F29E0F01550EA76EAA0EA76EA682A6B23E
:100D5000FED7A6940050F212020100013AEF39F0DA
:100D6000030EEA6E5A0EE96EEF500DE0060E016EAC
:100D7000006A002EFED7012EFBD77B0E006E002EE0
:100D8000FED7EF2EF3D7000C080E0501E96FE953EB
:100D90000CE0839AE851800B02E1839801D08388AC
:100DA000838AD890E837E907F2D70001000C8392D4
:100DB0008396E6C5E8F5E8DF8386000C0501E4517B
:100DC000070B4009E56FE66F0001F1DF0501E35114
:100DD0007F0B8009E56FE66F0001E9DF000C83827D
:100DE0008396E7C5E8F5D0DF8386000C0501E36B49
:100DF000E46B0001E3DF010E0201326FF80E316F88
:100E0000315302E132530AE00501E76B0001E7DFED
:100E100002013151D8B432073107F2D7000132EF65
:100E200007F08382838683940A0E03015A6F0001C0
:100E300097DF8384210E0501E66F0001B8DF2DC224
:100E4000E6F5B5DF130E0501E66F0001B0DF200EF9
:100E50000501E66F0001ABDF090E0501E66F000139
:100E6000A6DFC4D7080E0501E66F0001A0DF0C0E57
:100E70000501E66F00019BDF000C02013051C7083D
:100E800003E1800E306FE2D03051FC0803E1810EA7
:100E9000306FDCD03051E90803E1820E306FD6D0DC
:100EA0003051E20803E1830E306FD0D03051E408B6
:100EB00003E1840E306FCAD03051E00803E1850EA3
:100EC000306FC4D03051E50803E1860E306FBED0DC
:100ED0003051E70803E1870E306FB8D03051EA088F
:100EE00003E1880E306FB2D03051EB0803E1890E78
:100EF000306FACD03051E80803E18A0E306FA6D0D5
:100F00003051EF0803E18B0E306FA0D03051EE0866
:100F100003E18C0E306F9AD03051EC0803E18D0E56
:100F2000306F94D03051C40803E18E0E306F8ED0F4
:100F30003051C50803E18F0E306F88D03051C90899
:100F400003E1900E306F82D03051E60803E1910E3C
:100F5000306F7CD03051C60803E1920E306F76D0EE
:100F60003051F40803E1930E306F70D03051F60821
:100F700003E1940E306F6AD03051F20803E1950E10
:100F8000306F64D03051FB0803E1960E306F5ED0B5
:100F90003051F90803E1970E306F58D0303D03D03F
:100FA000980E306F53D03051D60803E1990E306F50
:100FB0004DD03051DC0803E19A0E306F47D03051EC
:100FC000F80803E19B0E306F41D03051A30803E1D4
:100FD0009C0E306F3BD03051D80803E19D0E306F2E
:100FE00035D03051D70803E19E0E306F2FD03051ED
:100FF000830803E19F0E306F29D03051E10803E1EF
:10100000A00E306F23D03051ED0803E1A10E306FF8
:101010001DD03051F30803E1A20E306F17D03051CC
:10102000FA0803E1A30E306F11D03051F10803E14B
:10103000A40E306F0BD03051D10803E1A50E306FF4
:1010400005D03051DF0802E1A60E306F00014EEFEF
:1010500008F083828396080E0501E86FE85310E0DC
:10106000839A030E006E002EFED7E751010B02E1BA
:10107000839801D08388838AD890E733E807EED736
:1010800083860001000C020130511F0802E38BD05F
:1010900006D030517F0803E20001EFD60201305143
:1010A0001F0801E380D03051A60801E27CD02E6BEE
:1010B0002E5104086AE330514F081EE33051E00F0F
:1010C000050DF350486B476F2E5147250501E76F1B
:1010D000000E020148210501E86F036EE751F2CFCF
:1010E000E9F5F29E000102EC00F00501E9BFF28E85
:1010F000E8CF2FF23DD0020130517F081EE330517E
:10110000B00F050DF350486B476F2E514725050171
:10111000E76F000E020148210501E86F036EE751F9
:10112000F2CFE9F5F29E000182EC00F00501E9BF83
:10113000F28EE8CF2FF21CD002013051A60818E33E
:101140003051800F050DF350486B476F2E514725E6
:101150000501E76F000E020148210501E86F6A0EE4
:10116000E725E96E010EE821EA6EEFCF2FF20201CA
:10117000010140AF03D0FF0E02012F1B2FC2E7F584
:1011800000012DDE02012E2B93D7010140BF05D0B7
:101190000501E76B00015DDF05D0FF0E0501E76F7C
:1011A000000157DF02010001D9EF08F0E6C530F277
:1011B0006AD7000C0501E751016AE65D03E2E6C566
:1011C00000F00CD0006A080EE86FE6370036E751F1
:1011D000005CD8B0006E0136E82FF7D70001000C94
:1011E0000150E3C5E6F5640E0501E76F0001E2DF9B
:1011F00000C0E3F50150300E08E10501E4A30ED074
:10120000E4B70CD0E4B9200E04D00501E497E499CA
:10121000E481012601509EA8FED7AD6EE3C5E6F538
:101220000A0EE76F0001C6DF00C0E3F50150300E83
:1012300008E10501E4B70BD0E4A109D0E4B9200E20
:101240000001012601509EA8FED7AD6E0501300EAB
:10125000E327E3519EA8FED7AD6E0001000C1E0EE1
:101260000501E36F010EE46F0001A8DD4C0E0501DE
:10127000E66F00019BDF430E0501E66F000196DF7C
:10128000440E0501E66F000191DF0C0E0501E36FCE
:10129000020EE46F000192DD03015A6B5A51000106
:1012A00002EC01F003015A2B006EE8CFE6F50001D5
:1012B0007DDF0A0E03015A5DF1E1180E0501E36FAF
:1012C000030EE46F00017ADD03015A6B5A510001ED
:1012D00010EC01F003015A2B006EE8CFE6F5000197
:1012E00065DF060E03015A5DF1E1030E0501E36FB0
:1012F000050EE46F000162DD03015A6B5A510001D3
:101300001CEC01F003015A2B006EE8CFE6F500015A
:101310004DDF0D0E03015A5DF1E184A432D00201CC
:101320002D3D03D003012DD00201010E2D27C80E43
:1013300003015A6F000114DD210E0501E66F000163
:1013400036DD2DC2E6F533DD03015A6B5A5100013B
:101350002BEC01F003015A2B006E00509EA8FED723
:10136000AD6E050E5A5DF2E12DC2E3F51B0E0501CF
:10137000E46F000135DF200E9EA8FED7AD6E03019D
:10138000CCD784A233D002012D518008D8A002D03E
:1013900003012CD0010E2D5FC80E03015A6F00010E
:1013A000DFDC210E0501E66F000101DD2DC2E6F54F
:1013B000FEDC03015A6B5A5100012BEC01F00301D2
:1013C0005A2B006E00509EA8FED7AD6E050E5A5DDA
:1013D000F2E12DC2E3F51B0E0501E46F000100DF11
:1013E000200E9EA8FED7AD6E0301CBD7A96A2DC2F1
:1013F000A8FFA69CA69EA684F2CF00F0F29E0F0145
:10140000550EA76EAA0EA76EA682A6B2FED7A69408
:101410000050F212000105DD3EEF39F00501E36BEB
:10142000E2C5E4F50001CADC0501E36BE35100010C
:1014300038EC01F00501E32B006EE66F0001B6DE2B
:101440000E0E0501E35DF2E10001000C8088070E3D
:101450000301646F643D01D008D080940000000057
:101460008084000000006407F5D7000E016E0001C3
:10147000000C0501F96B070EFA6FFA3D01D01FD081
:10148000F8C500F0FA51016E04E0D8900032012E48
:10149000FCD700A0809800B08088000080948084F1
:1014A00080A60BD0010E006EFA51016E04E0D890B8
:1014B0000036012EFCD70050F913FA07DED7F9C524
:1014C00001F00001000CFF0E0501F86F0001D1DFF3
:1014D0005AC5F8F5CEDF5CC560F50501616B5CC5EA
:1014E000F8F50001C6DF5BC5F8F5C3DF5EC560F542
:1014F0000501616B5EC5F8F50001BBDF5DC5F8F560
:10150000B8DF5FC5F8F5B5DFFF0E0501F86F000124
:10151000B0DFFF0E0501F86F0001ABDF01C04AF23A
:1015200002014AC201F00001000C05015CBF10D0AD
:101530000F0E006E5B3900160A0E005C03E2300EDF
:10154000002602D05C51002600509EA8FED7AD6E4A
:101550000F0E5B170A0E5B5D02E2300E02D05C9F3D
:101560005C515B275B519EA8FED7AD6E0001000C5D
:101570000201586B576B566B556BFF0E0501F86FE8
:10158000000177DF64C3F8F574DFFF0E0501F86F23
:1015900000016FDFFF0E0501F86F00016ADFFF0E2B
:1015A0000501F86F000165DFFF0E0501F86F00010E
:1015B00060DFFF0E0501F86F00015BDFFF0E050124
:1015C000F86F000156DFFF0E0501F86F000151DFD3
:1015D000FF0E0501F86F00014CDF0201586B576BDD
:1015E000566B01C055F257C258F256C257F255C257
:1015F00056F2556BFF0E0501F86F00013ADF0150FE
:1016000002015527000E56235723582357C258F27C
:1016100056C257F255C256F2556BFF0E0501F86FD0
:10162000000127DF015002015527000E56235723E2
:10163000582357C258F256C257F255C256F2556B4C
:10164000FF0E0501F86F000114DF0150020155275C
:10165000000E56235723582355C200F056C201F0FE
:1016600057C202F058C203F00001000C010140A56E
:1016700010D00301646B6451000148EC01F00301D8
:10168000642B006E00509EA8FED7AD6E070E645D01
:10169000F2E10501E36B040EE46F0001DEEC06F0FD
:1016A0000301646B6451000154EC01F00301642BED
:1016B000006EE8CFE6F5000179DD0D0E0301645DF3
:1016C000F1E180820A0E5A6F5A3D01D005D0000127
:1016D000BDDE03015A07F8D78092400E05015A6F0C
:1016E0005C6B5B6B5E6B5D6B950E5F6F0001EBDEA1
:1016F00001C05BF303015B2D01D002D00001B6D71E
:101700000001A4DEA3DE480E05015A6F5C6B5B6B23
:10171000010E5E6FAA0E5D6F870E5F6F0001D3DE54
:1017200001C05BF3010140A51BD00301646B645150
:10173000000163EC01F00301642B006E00509EA8D1
:10174000FED7AD6E060E645DF2E15BC35BF5570E2E
:1017500005015C6F0001E9DE200E9EA8FED7AD6E8C
:1017600003015B2D40D0FF0E0501F86F000181DE03
:1017700001C05BF3FF0E0501F86F00017ADE01C0C6
:101780005BF3FF0E0501F86F000173DE01C05DF32E
:10179000010140A50BD05DC35BF5570E05015C6FE1
:1017A0000001C3DE200E9EA8FED7AD6EFF0E050120
:1017B000F86F00015EDE01C05EF3010140A50BD0B1
:1017C0005EC35BF5570E05015C6F0001AEDE200EB7
:1017D0009EA8FED7AD6E03015D2D05D05E51AA080F
:1017E00002E1010E5C6F5C5319E10501E36B040E2D
:1017F000E46F0001DEEC06F00301646B645100014C
:1018000070EC01F00301642B006EE8CFE6F50001F7
:10181000CDDC0C0E0301645DF1E12DD17A0E646F15
:101820000001A6DE03C062F302C061F301C060F3F1
:1018300000C05FF3010140A530D00301646B645127
:1018400000017FEC01F00301642B006E00509EA8A4
:10185000FED7AD6E070E645DF2E162C35BF5570E15
:1018600005015C6F000161DE61C35BF5570E050188
:101870005C6F00015ADE60C35BF5570E05015C6FBB
:10188000000153DE5FC35BF5570E05015C6F00017D
:101890004CDE200E9EA8FED7AD6E0301646B60C3C4
:1018A00065F361C366F3676B645307E165518008B4
:1018B00004E1663D02D0675301E0B0D7770E050121
:1018C0005A6F5C6B5B6B5E6B5D6BFF0E5F6F000155
:1018D000FADD01C05DF3690E05015A6F400E5C6FC1
:1018E0005B6B5E6B5D6BFF0E5F6F0001ECDD01C03B
:1018F0005EF303015D51010803E25E5301E0DED7B0
:101900007A0E646F000134DE03C062F302C061F33B
:1019100001C060F300C05FF3010140A530D00301B6
:10192000646B645100018DEC01F00301642B006EC7
:1019300000509EA8FED7AD6E070E645DF2E162C353
:101940005BF5570E05015C6F0001EFDD61C35BF5D0
:10195000570E05015C6F0001E8DD60C35BF5570EB3
:1019600005015C6F0001E1DD5FC35BF5570E05010A
:101970005C6F0001DADD200E9EA8FED7AD6E02017D
:10198000996B030162AD03D00201992B0301646BD3
:1019900060C365F361C366F3676B645307E1655128
:1019A000800804E1663D02D0675301E0A9D7010138
:1019B00040A51CD00301646B645100019BEC01F055
:1019C0000301642B006E00509EA8FED7AD6E060E7C
:1019D000645DF2E199C25BF5570E05015C6F000191
:1019E000A4DD200E9EA8FED7AD6E01010201995321
:1019F00024E1030163516408D8B002D002011DD074
:101A0000632B0501E36B040EE46F0001DEEC06F0CE
:101A10000301646B64510001A8EC01F00301642B25
:101A2000006EE8CFE6F50001D6EC08F00C0E0301DD
:101A3000645DF0E143D71CD00201992D1AD0050155
:101A4000E36B040EE46F0001DEEC06F00301646B4F
:101A500064510001B7EC01F00301642B006EE8CF84
:101A6000E6F50001D6EC08F00C0E0301645DF0E130
:101A7000020151D003017A0E646F000179DD03C0C9
:101A800062F302C061F301C060F300C05FF30101C3
:101A900040A530D00301646B64510001C6EC01F035
:101AA0000301642B006E00509EA8FED7AD6E070E9A
:101AB000645DF2E162C35BF5570E05015C6F0001E6
:101AC00034DD61C35BF5570E05015C6F00012DDD50
:101AD00060C35BF5570E05015C6F000126DD5FC337
:101AE0005BF5570E05015C6F00011FDD200E9EA8FF
:101AF000FED7AD6E0301646B60C365F361C366F32B
:101B0000676B645307E16551800804E1663D02D0CC
:101B1000675301E0B0D70501E36B050EE46F0001E8
:101B2000DEEC06F0770E05015A6F5C6B5B6B5E6B4B
:101B30005D6BFF0E5F6F0001C6DC01C05BF3690ED9
:101B400005015A6F400E5C6F5B6B5E6B5D6BFF0E49
:101B50005F6F0001B8DC01C05BF3010140A51BD041
:101B60000301646B64510001D4EC01F00301642BA8
:101B7000006E00509EA8FED7AD6E080E645DF2E1C7
:101B80005BC35BF5570E05015C6F0001CEDC200ED8
:101B90009EA8FED7AD6E03015B51050802E109D096
:101BA00005D05B5303E00201B6D70301000E016EBE
:101BB0004FD0010140A510D00301646B64510001B6
:101BC000E2EC01F00301642B006E00509EA8FED7EA
:101BD000AD6E090E645DF2E1FF0E0501F86F0001C4
:101BE00048DC410E05015A6F5C6B5B6B5E6B5D6B95
:101BF000FF0E5F6F000167DC015222E00501E36B1D
:101C0000040EE46F0001DEEC06F00301646B645126
:101C10000001EFEC01F00301642B006EE8CFE6F564
:101C20000001D6EC08F0090E0301645DF0E1050146
:101C3000E36B050EE46F0001DEEC06F00301B9D79B
:101C4000FF0E0501F86F000114DC010E016E0301A7
:101C50000001E0EF39F0F0C5F8F50BDCF2C5F6F560
:101C60000501F76BF2C5F8F5000103DCF1C5F8F5E5
:101C700000DCF4C5F6F50501F76BF4C5F8F50001D5
:101C800039EC0AF0F3C5F8F539EC0AF0F5C5F8F5CA
:101C900039EC0AF0FF0E0501F86F000139EC0AF08B
:101CA000000C020199530DE1D890E4C5E5F5E3C5B8
:101CB000E4F5E2C5E3F50501E26BE337E437E53728
:101CC00002018092E4C5ECF5E5C5EDF50501E2C53C
:101CD000EEF5E3C5EFF5510EF06FE5C5F2F5E4C59D
:101CE000F1F5E3C5F4F5E2C5F3F5FF0EF56F00017C
:101CF000B2DFFF0E0501F86F000139EC0AF001C0F8
:101D0000EAF50501EA5303E00001F3D70501FF0EF0
:101D1000F86F000139EC0AF00150FE08D8B402D087
:101D20000501F5D70501E96BE86BE951010819E3F5
:101D3000E7C503F0E651E62BD8B4E72BEB6F03C001
:101D4000ECF5FF0EF86F000139EC0AF0ECC5EAFF84
:101D5000EBC5E9FF01C0EFFF0501E82BD8B4E92B83
:101D6000E4D7FF0EF86F000139EC0AF08082000E14
:101D7000016E000C0501EE6BEF6B010EF06FDA6A7D
:101D8000D96A050EF36FE60EF26F050EEA6EEA0EE3
:101D9000E96EF3C5E2FFF2C5E1FFF0C5F1F5D890B9
:101DA000E550EE02F350EE23F450EF23F12FF7D776
:101DB000EEC5DEFFEFC5EEF5EF6BD8B0EF2BF22BE3
:101DC000D8B4F32BF02BF0510508DFE10001000C33
:101DD00005015A515C03F3CF01F0F4CF00F05D032D
:101DE000F35000265B515C03F3500020026E0001AB
:101DF000000C006A016A026A036A0501FB6BFC6B56
:101E0000FD6BFE6BFA51F911F811F7112CE0200E61
:101E1000FF6FD890F337F437F537F637FB37FC37D9
:101E2000FD37FE37FA51FE5D08E1F951FD5D05E130
:101E3000F851FC5D02E1F751FB5D0FE3F751FB5FE9
:101E4000F851D8A0F83DFC5FF951D8A0F93DFD5FED
:101E5000FA51D8A0FA3DFE5FD8800036013602362E
:101E60000336FF2FD6D7050EEA6EFB0EE96E000192
:101E7000000C8092FF0E0501F86F000139EC0AF0AA
:101E8000500E05015A6F5C6B5B6B020E5E6F5D6BF3
:101E9000FF0E5F6F000163EC0AF0015201E0EAD728
:101EA000FF0E0501F86F000139EC0AF0FF0E050185
:101EB000F86F000139EC0AF080820501E56BE46BF4
:101EC000E36BE26B030EE76F5A0EE66F0001E9DE8B
:101ED00023C55CF20201596B5A6B5B6B05015B6BAE
:101EE0005BC503F022C502F0006A016A00500201DE
:101EF000592701505A2302505B2303505C230501EC
:101F00005C6B5B6B5CC503F05BC502F021C501F047
:101F1000006A00500201592701505A2302505B23E6
:101F200003505C2320C500F0016A026A036A005076
:101F3000592701505A2302505B2303505C230101AF
:101F400040A53BD005015A6B5A510001FCEC01F051
:101F500005015A2B006E00509EA8FED7AD6E060EEE
:101F60005A5DF2E15CC25BF5570E5C6F000195ECC7
:101F70000AF05BC25BF5570E05015C6F000195EC42
:101F80000AF05AC25BF5570E05015C6F000195EC33
:101F90000AF059C25BF5570E05015C6F000195EC24
:101FA0000AF0200E9EA8FED7AD6E0A0E9EA8FED7A0
:101FB000AD6E0D0E9EA8FED7AD6E5CC2E5F55BC2A0
:101FC000E4F55AC2E3F559C2E2F5030E0501E76FE5
:101FD0005A0EE66F000165DE05015C6B5B6B66C344
:101FE00060F55F6B0301655105015F250201616FBB
:101FF000000E050160210201626F000E05015B21E8
:102000000201636F000E05015C210201646F010192
:1020100040A53CD005015A6B5A5100010BEC02F06F
:1020200005015A2B006E00509EA8FED7AD6E070E1C
:102030005A5DF2E164C25BF5570E5C6F000195ECEE
:102040000AF063C25BF5570E05015C6F000195EC69
:102050000AF062C25BF5570E05015C6F000195EC5A
:102060000AF061C25BF5570E05015C6F000195EC4B
:102070000AF0200E9EA8FED7AD6E0A0E9EA8FED7CF
:10208000AD6E0D0E9EA8FED7AD6E010167C34BF27B
:1020900040A523D005015A6B5A5100011AEC02F0F9
:1020A00005015A2B006E00509EA8FED7AD6E090E9A
:1020B0005A5DF2E14BC25BF5570E5C6F000195EC87
:1020C0000AF0200E9EA8FED7AD6E0A0E9EA8FED77F
:1020D000AD6E0D0E9EA8FED7AD6E050169C360F50D
:1020E0005F6B0301685105015F2502014F6F000E10
:1020F000050160210201506F010140A52CD00501AE
:102100005A6B5A5100012AEC02F005015A2B006E5D
:1021100000509EA8FED7AD6E060E5A5DF2E150C289
:102120005BF5570E5C6F000195EC0AF04FC25BF552
:10213000570E05015C6F000195EC0AF0200E9EA879
:10214000FED7AD6E0A0E9EA8FED7AD6E0D0E9EA8F0
:10215000FED7AD6E01016AC34CF240A523D0050144
:102160005A6B5A51000139EC02F005015A2B006EEE
:1021700000509EA8FED7AD6E060E5A5DF2E14CC22D
:102180005BF5570E5C6F000195EC0AF0200E9EA8DF
:10219000FED7AD6E0A0E9EA8FED7AD6E0D0E9EA8A0
:1021A000FED7AD6E02014F5159255D6F50515A2136
:1021B0005E6F000E5B215F6F000E5C21606F01019E
:1021C00040A53BD005015A6B5A51000147EC02F083
:1021D00005015A2B006E00509EA8FED7AD6E090E69
:1021E0005A5DF2E160C25BF5570E5C6F000195EC41
:1021F0000AF05FC25BF5570E05015C6F000195ECBC
:102200000AF05EC25BF5570E05015C6F000195ECAC
:102210000AF05DC25BF5570E05015C6F000195EC9D
:102220000AF0200E9EA8FED7AD6E0A0E9EA8FED71D
:10223000AD6E0D0E9EA8FED7AD6E60C2E9F55FC211
:10224000E8F55EC2E7F55DC2E6F564C2EDF563C28E
:10225000ECF562C2EBF561C2EAF500018BDD03C06B
:1022600070F202C06FF201C06EF200C06DF20101A7
:1022700040A53BD005015A6B5A51000157EC02F0C2
:1022800005015A2B006E00509EA8FED7AD6E100EB1
:102290005A5DF2E170C25BF5570E5C6F000195EC80
:1022A0000AF06FC25BF5570E05015C6F000195ECFB
:1022B0000AF06EC25BF5570E05015C6F000195ECEC
:1022C0000AF06DC25BF5570E05015C6F000195ECDD
:1022D0000AF0200E9EA8FED7AD6E0A0E9EA8FED76D
:1022E000AD6E0D0E9EA8FED7AD6E050171C360F5F3
:1022F0005F6B0301705105015F250201516F000EF4
:10230000050160210201526F010140A52BD005019A
:102310005A6B5A5100016BEC02F005015A2B006E0A
:1023200000509EA8FED7AD6E070E5A5DF2E152C274
:102330005BF5570E5C6F000195EC0AF051C25BF53E
:10234000570E05015C6F000195EC0AF0200E9EA867
:10235000FED7AD6E0A0E9EA8FED7AD6E0D0E9EA8DE
:10236000FED7AD6E05016CC360F55F6B03016B5169
:1023700005015F250201536F000E05016021020176
:10238000546F010140A52BD005015A6B5A51000131
:102390007AEC02F005015A2B006E00509EA8FED781
:1023A000AD6E0A0E5A5DF2E154C25BF5570E5C6FDA
:1023B000000195EC0AF053C25BF5570E05015C6F06
:1023C000000195EC0AF0200E9EA8FED7AD6E0A0E15
:1023D0009EA8FED7AD6E0D0E9EA8FED7AD6E050170
:1023E000E96BE86BE76B4BC2E6F564C2EDF563C2DF
:1023F000ECF562C2EBF561C2EAF50001BBDC03C09B
:1024000074F202C073F201C072F200C071F20201F4
:10241000535303E15453D8B4CBD0515303E1525337
:10242000D8B4C6D0499152C25BF551C25AF50501E4
:102430005D6B4CC25CF50001CBDC015002015D25F7
:10244000796F02505E217A6F000E5F217B6F000E64
:1024500060217C6F010140A53BD005015A6B5A51A8
:1024600000018BEC02F005015A2B006E00509EA873
:10247000FED7AD6E0B0E5A5DF2E17CC25BF5570ED6
:102480005C6F000195EC0AF07BC25BF5570E05010D
:102490005C6F000195EC0AF07AC25BF5570E0501FE
:1024A0005C6F000195EC0AF079C25BF5570E0501EF
:1024B0005C6F000195EC0AF0200E9EA8FED7AD6E71
:1024C0000A0E9EA8FED7AD6E0D0E9EA8FED7AD6E6D
:1024D0000201533505015A6F0201543505015B6F46
:1024E0005A375B375A375B375A375B375A375B3760
:1024F000E00E5A17F66BF56B5BC5F4F55AC5F3F5AC
:1025000064C2FAF563C2F9F562C2F8F561C2F7F583
:1025100000016FDC0050020179257D6F01507A21A6
:102520007E6F02507B217F6F03507C21806F010101
:1025300040A53CD005015A6B5A5100019CEC02F0B9
:1025400005015A2B006E00509EA8FED7AD6E0E0EF0
:102550005A5DF2E180C25BF5570E5C6F000195ECAD
:102560000AF07FC25BF5570E05015C6F000195EC28
:102570000AF07EC25BF5570E05015C6F000195EC19
:102580000AF07DC25BF5570E05015C6F000195EC0A
:102590000AF0200E9EA8FED7AD6E0A0E9EA8FED7AA
:1025A000AD6E0D0E9EA8FED7AD6E0101EDD10201FC
:1025B000498181C368F20201656B666B676B050137
:1025C0005B6B5BC503F080C302F0006A016A0050D8
:1025D00002016527015066230250672303506823D8
:1025E00005015C6B5B6B5CC503F05BC502F07FC3F0
:1025F00001F0006A00500201652701506623025075
:102600006723035068237EC300F0016A026A036AED
:10261000005065270150662302506723035068234A
:10262000010140A53BD005015A6B5A510001AFECA6
:1026300002F005015A2B006E00509EA8FED7AD6E29
:102640000A0E5A5DF2E168C25BF5570E5C6F00013D
:1026500095EC0AF067C25BF5570E05015C6F00014F
:1026600095EC0AF066C25BF5570E05015C6F000140
:1026700095EC0AF065C25BF5570E05015C6F000131
:1026800095EC0AF0200E9EA8FED7AD6E0A0E9EA80D
:10269000FED7AD6E0D0E9EA8FED7AD6E89C36CF24F
:1026A0000201696B6A6B6B6B05015B6B5BC503F0C9
:1026B00088C302F0006A016A0050020169270150D4
:1026C0006A2302506B2303506C2305015C6B5B6B28
:1026D0005CC503F05BC502F087C301F0006A0050DF
:1026E0000201692701506A2302506B2303506C23B7
:1026F00086C300F0016A026A036A0050692701502C
:102700006A2302506B2303506C23010140A53BD088
:1027100005015A6B5A510001C0EC02F005015A2B19
:10272000006E00509EA8FED7AD6E110E5A5DF2E10C
:102730006CC25BF5570E5C6F000195EC0AF06BC242
:102740005BF5570E05015C6F000195EC0AF06AC25B
:102750005BF5570E05015C6F000195EC0AF069C24C
:102760005BF5570E05015C6F000195EC0AF0200E39
:102770009EA8FED7AD6E0A0E9EA8FED7AD6E0D0EBA
:102780009EA8FED7AD6E68C2E9F567C2E8F566C2DD
:10279000E7F565C2E6F50501ED6BEC6BEB6B4CC242
:1027A000EAF50001BAEC0EF0005002015D25796FE8
:1027B00001505E217A6F02505F217B6F03506021D0
:1027C0007C6F010140A53BD005015A6B5A510001B5
:1027D0008BEC02F005015A2B006E00509EA8FED72C
:1027E000AD6E0B0E5A5DF2E17CC25BF5570E5C6F6D
:1027F000000195EC0AF07BC25BF5570E05015C6F9A
:10280000000195EC0AF07AC25BF5570E05015C6F8A
:10281000000195EC0AF079C25BF5570E05015C6F7B
:10282000000195EC0AF0200E9EA8FED7AD6E0A0EB0
:102830009EA8FED7AD6E0D0E9EA8FED7AD6E7CC2D3
:10284000E9F57BC2E8F57AC2E7F579C2E6F564C23C
:10285000EDF563C2ECF562C2EBF561C2EAF5000189
:10286000BAEC0EF003C084F202C083F201C082F21F
:1028700000C081F2010140A53BD005015A6B5A51BD
:102880000001D4EC02F005015A2B006E00509EA806
:10289000FED7AD6E0B0E5A5DF2E184C25BF5570EAA
:1028A0005C6F000195EC0AF083C25BF5570E0501E1
:1028B0005C6F000195EC0AF082C25BF5570E0501D2
:1028C0005C6F000195EC0AF081C25BF5570E0501C3
:1028D0005C6F000195EC0AF0200E9EA8FED7AD6E4D
:1028E0000A0E9EA8FED7AD6E0D0E9EA8FED7AD6E49
:1028F00002014B5179257D6F000E7A217E6F000E0B
:102900007B217F6F000E7C21806F010140A53CD0B0
:1029100005015A6B5A5100019CEC02F005015A2B3B
:10292000006E00509EA8FED7AD6E0E0E5A5DF2E10D
:1029300080C25BF5570E5C6F000195EC0AF07FC218
:102940005BF5570E05015C6F000195EC0AF07EC245
:102950005BF5570E05015C6F000195EC0AF07DC236
:102960005BF5570E05015C6F000195EC0AF0200E37
:102970009EA8FED7AD6E0A0E9EA8FED7AD6E0D0EB8
:102980009EA8FED7AD6E01017CC278F27BC277F2C1
:102990007AC276F279C275F20201615307E162519F
:1029A000020804E1635302E1645312E005015A6B2B
:1029B0005A510001E5EC02F005015A2B006E00505F
:1029C0009EA8FED7AD6E190E5A5DF2E1FF0002011E
:1029D0000001F6EF39F0030E03015D5F0AE3030E19
:1029E000EA6E5D0EE96EEF5004E001D000D0EF2EEC
:1029F000FDD70001000C0301776B070E786F783D5F
:102A000001D01ED0829676C300F07851016E04E0AA
:102A1000D8900032012EFCD700A0829A00B0828AA2
:102A2000828682A80BD0010E006E7851016E04E000
:102A3000D8900036012EFCD7005077137807DFD7E7
:102A400077C301F00001000C0301706B716B726BB6
:102A5000736B746B756B82946CC376F30001CBDF80
:102A60006DC376F3C8DF6EC376F3C5DF0301716B08
:102A700001C070F36FC376F30001BDDF0301736B18
:102A800001C072F3766B76517211746F70517311CD
:102A9000756F828474C301F075C302F00001000CED
:102AA0008284819C020E03015A6FF90E5D6F000152
:102AB00092DF03015A2FF9D7818C020E5A6FF90E5B
:102AC0005D6F000188DF03015A2FF9D7020E6C6F8A
:102AD0000B0E6D6FA00E6E6F6F6F0001B5DF020EF3
:102AE00003016C6F030E6D6F300E6E6FD40E6F6F3F
:102AF0000001AADF280E0101516F020E03016C6F65
:102B00000B0E6D6F51C16EF351C16FF300019CDF6D
:102B10000CEF3AF0E9500501EB6F3B0EF26F9A0EA5
:102B2000F16FCA0EF06FEF6B0A0EED6FEAC5F6F5A6
:102B3000E9C5F5F5E8C5F4F5E7C5F3F5F2C5FAF52D
:102B4000F1C5F9F5F0C5F8F5EFC5F7F50001F9ECB9
:102B50000EF00150EFCFE7F5ECCFE8F5ECCFE9F55B
:102B6000ECCFEAF5005213E10501ED51010AD8A4BA
:102B700002D000010CD0EB510CE00F0BED5D01E039
:102B80000EE2EBBF0CD0EBBD04D0200E03D005014C
:102B9000EB6B300E002600509EA8FED7AD6EF2C53E
:102BA000F6F5F1C5F5F5F0C5F4F5EFC5F3F5FA6BFB
:102BB000F96BF86B0A0EF76F0001F9EC0EF003C029
:102BC000F2F502C0F1F501C0F0F500C0EFF5050126
:102BD000ED2FACD70001000C0150E4C5E6F5640E02
:102BE0000501E76F0001DAEC08F000C0E4F50150E0
:102BF000300E08E10501E5A310D0E5B70ED0E5B928
:102C0000200E04D00501E597E599E581012601C074
:102C1000E6F50001D6EC08F00501E4C5E6F50A0E7C
:102C2000E76F0001DAEC08F000C0E4F50150300E67
:102C300008E10501E5B70BD0E5A109D0E5B9200E03
:102C40000001012601C0E6F5D6EC08F00501300EC2
:102C5000E427E4C5E6F50001D6EC08F0000CEACF65
:102C6000EAF5E9CFE9F50501E339F009E56FE52774
:102C7000E20FE66F320FE86FE3510F0BE627E6270E
:102C8000E827E90FE76FE727E727E2390F0BE72788
:102C9000E827E737E837E81FE837E2510F0BE82766
:102CA000E537070EE46F0A0EE707E827FDE3E607BE
:102CB000E727FDE3E507E627FDE3E407E527FDE376
:102CC000050EEA6EE40EE96E070EE915E99DE926A8
:102CD000E80EE95CD8B4E98DEF50006E08E1E9BD7B
:102CE00006D0E9B90CD0E9B702D0200E03D0E987AD
:102CF000E999300E002600509EA8FED7AD6EEE502A
:102D0000E9ADE6D70001000C05017B6B01014B6BBF
:102D10004A6B416B426B0501676B666B656B646B5D
:102D20000101466B03015A2D1ED00501E36B040E11
:102D3000E46F0001DEEC06F00501E26BE2510001F8
:102D4000FAEC02F00501E22B006EE66F0001D6EC12
:102D500008F00B0E0501E25DF1E1E36B050EE46F97
:102D60000001DEEC06F0020149A110D060C263F55B
:102D70005FC262F55EC261F55DC260F56CC26BF563
:102D80006BC26AF56AC269F569C268F57CC27AF5F8
:102D90007BC279F57AC278F579C277F50501736B54
:102DA000726B716B706B020149A10FD04B51050121
:102DB0007725816F000E7821826F000E7921836F55
:102DC000000E7A21846F32D0020149B12FD05335E1
:102DD0000501E26F020154350501E36FE237E33785
:102DE000E237E337E237E337E237E337E00EE21763
:102DF000F66BF56BE3C5F4F5E2C5F3F564C2FAF5DD
:102E000063C2F9F562C2F8F561C2F7F50001F9ECA9
:102E10000EF0005005017725816F01507821826FF7
:102E200002507921836F03507A21846F7AC55FF550
:102E300079C55EF578C55DF577C55CF5050181510D
:102E40005C5D0BE182515D5D08E183515E5D05E1F2
:102E500084515F5DD8B4EFEF1CF0010140A595D01F
:102E60000501E26BE251000108EC03F00501E22BE1
:102E7000006E00509EA8FED7AD6E0A0EE25DF2E134
:102E8000410EE96E5FC5EAF55EC5E9F55DC5E8F599
:102E90005CC5E7F500013EDE200E9EA8FED7AD6EB4
:102EA0000501E26BE251000118EC03F00501E22B91
:102EB000006E00509EA8FED7AD6E080EE25DF2E1F6
:102EC000410EE96E6FC5EAF56EC5E9F56DC5E8F529
:102ED0006CC5E7F500011EDE200E9EA8FED7AD6E84
:102EE0000501E26BE251000127EC03F00501E22B42
:102EF000006E00509EA8FED7AD6E090EE25DF2E1B5
:102F0000410EE96E73C5EAF572C5E9F571C5E8F5DC
:102F100070C5E7F50001FEDD200E9EA8FED7AD6E60
:102F200005017B51040DF350036A920FE96E050E03
:102F30000320EA6EEFCFE2F5ECCFE3F5ECCFE4F55A
:102F4000ECCFE5F5E66BE651000136EC03F0050148
:102F5000E62B006E00509EA8FED7AD6E090EE65D12
:102F6000F2E1410EE96EE5C5EAF5E4C5E9F5E3C530
:102F7000E8F5E2C5E7F50001CDDD0A0E9EA8FED713
:102F8000AD6E0D0E9EA8FED7AD6E05016C530BE124
:102F90006D51020808E16E5306E16F5304E1736B53
:102FA000726B716B706B5FC5E5F55EC5E4F55DC571
:102FB000E3F55CC5E2F5030EE76F5C0EE66F00011A
:102FC00051EC0EF073C56FF572C56EF571C56DF5F8
:102FD00070C56CF505016C5309E16D51020806E1FD
:102FE0006E5304E16F53D8B4E5EF1CF05C0E6C2512
:102FF000E96E030E6D21EA6EEF507F0818E20101C1
:1030000040A511D00501E26BE251000146EC03F04E
:103010000501E22B006E00509EA8FED7AD6E040E97
:10302000E25DF2E10101DBEF1CF01CD305010B0EA8
:103030006C25E26F000E6D21E36F000E6E21E46FD0
:10304000000E6F21E56F5C0EE225E96E030EE321B1
:10305000EA6EEF500C0B0C0818E1010140A511D0ED
:103060000501E26BE251000151EC03F00501E22B96
:10307000006E00509EA8FED7AD6E040EE25DF2E138
:103080000101DBEF1CF0EED205015C0E6C25E96E50
:10309000030E6D21EA6EEF52D8A490D0FF0EE76FB9
:1030A0000001EFEC06F005017B51000868E2010128
:1030B00040A510D00501E26BE25100015CEC03F089
:1030C0000501E22B006E00509EA8FED7AD6E050EE6
:1030D000E25DF2E105017B07010E010142270501D6
:1030E0007B51040DF350036A920FE96E050E032025
:1030F000EA6EEFCF00F0ECCF01F0ECCF02F0ECCFB6
:1031000003F003C073F502C072F501C071F500C091
:1031100070F57B51040DF350036ABA0FE96E050E8A
:103120000320EA6EEFCF00F0ECCF01F0ECCF02F01D
:10313000ECCF03F003C07AF502C079F501C078F551
:1031400000C077F5200E7027000E712372237323C1
:10315000705313E17151020810E172530EE1735381
:103160000CE1010E7727D8B0782BD8B4792BD8B4DE
:103170007A2B736B726B716B706B15D61ED07B5391
:103180001CE1010140A510D00501E26BE2510001F4
:1031900067EC03F00501E22B006E00509EA8FED7FD
:1031A000AD6E050EE25DF2E1040E0501E26F000175
:1031B0000EEC0AF031EF20F0050156D20B0E6C2513
:1031C000E26F000E6D21E36F000E6E21E46F000EC2
:1031D0006F21E56F5C0EE225E96E030EE321EA6ED6
:1031E000EF501C0B1008D8A4D2D15C0E6C25E96EF0
:1031F000030E6D21EA6EEF502E0803E10101DBEFB3
:103200001CF003015A5304E10101472B16D00301BE
:103210005A51020812E10101462B4651455D0DE16C
:10322000010E4A254C6F000E4B214D6F409B010E45
:1032300003015A6F000168D5010105017B51040D9E
:10324000F350036A920FE96E050E0320EA6E6CC517
:10325000EFFF6DC5ECFF6EC5ECFF6FC5ECFF7B515A
:10326000040DF350036ABA0FE96E050E0320EA6EEF
:103270005CC5EFFF5DC5ECFF5EC5ECFF5FC5ECFF15
:103280007B2B0101412B036A4151BF0FE96E020EF6
:103290000320EA6E7BC5EFFF426B03015A5103081E
:1032A000D8A4C2D00101455302E1010E456F462B5F
:1032B0004551465DD8A08ED005017B5100083DE206
:1032C000050EEA6E850EE96EF2CFE2F5F29E000E73
:1032D000000172EC03F00A000900F550EE6E0009DF
:1032E000FBE10501E2BFF28E03015B6B5B51080855
:1032F00023E0036A5B51850F016E050E0322030173
:103300005B5105016C25E46F000E6D21E56F000E29
:103310006E21000E6F215C0EE425E96E030EE5219F
:10332000EA6EEFCFE8F503C0EAFF01C0E9FFE8C5A8
:10333000EFFF03015B2BDAD70501E36B50C1E4F526
:103340000001DEEC06F001015053D8B4408F50511B
:103350004525036A9A0FE96E020E0320EA6EEFCF4D
:10336000E3F5E3C5E4F5130E0501E56F000134DC78
:10337000200E0501E66F0001D6EC08F07BC57CF558
:1033800005017C5308E02E0EE66F0001D6EC08F034
:1033900005017C07F6D75C0EE66F0001D6EC08F05D
:1033A000050EEA6E850EE96E000EEF1010E0EACF12
:1033B000E3F5E9CFE2F5EFCFE6F5D6EC08F0E3C5AB
:1033C000EAFFE2C5E9FFE92AD8B4EA2AEDD701010C
:1033D000409F502B030E4525465D03E04751465D57
:1033E00022E10501E36B040EE46F0001DEEC06F060
:1033F0000501E26BE25100017BEC03F00501E22BD9
:10340000006EE66F0001D6EC08F0080E0501E25DE3
:10341000F1E19AC2E4F51B0EE56F0001ECEC15F04A
:1034200031EF20F0010103015A2D02D041C145F1D5
:10343000150E05016C25E26F000E6D21E36F000E85
:103440006E21000E6F215C0EE225E96E030EE32172
:10345000EA6EEF50E66FEB6BEC6BED6B140E6C25C8
:10346000EF6F000E6D21F06F000E6E21000E6F21C8
:103470005C0EEF25E96E030EF021EA6EEF50F46B5F
:10348000F36F006A016A0050EB257D6F0150EC215B
:103490007E6FF351ED217F6FF451E621806F1B0E9B
:1034A0006C25E26F000E6D21E36F000E6E21000EA1
:1034B0006F215C0EE225E96E030EE321EA6EEF5008
:1034C000E86BE76BE66FEB6B1A0E6C25EF6F000E87
:1034D0006D21F06F000E6E21000E6F215C0EEF2546
:1034E000E96E030EF021EA6EEF50EB25006E000E40
:1034F000E621016E000EE721026E000EE821036E48
:1035000000507D2701507E2302507F2303508023EB
:10351000020E7D5F000E7E5B7F5B805B80C5E9F500
:103520007FC5E8F57EC5E7F57DC5E6F5ED6BEC6B8F
:10353000EB6B4BC2EAF50001BAEC0EF003C07AF572
:1035400002C079F501C078F500C077F502017D5120
:103550000501772702017E510501782302017F5181
:10356000050179230201805105017A23020149A155
:1035700007D04B510501775F000E785B795B7A5B72
:103580000501736B726B716B706B0DD46DD00301A1
:103590005A5369E1010140A51ED00501E26BE251D9
:1035A000000189EC03F00501E22B006E00509EA89B
:1035B000FED7AD6E090EE25DF2E1100EE96E49C173
:1035C000E3F548C1E2F500012FEC16F0200E9EA8AD
:1035D000FED7AD6E010140A51BD00501E26BE251A3
:1035E000000196EC03F00501E22B006E00509EA84E
:1035F000FED7AD6E0B0EE25DF2E141C1E3F51B0EAD
:10360000E46F0001F0EC08F0200E9EA8FED7AD6E2E
:1036100005017B5321E0010142530FE04251415D1E
:10362000036ABF0FE96E020E0320EA6EEF50050138
:103630007B5D04E20101422BF1D7050101014251FA
:10364000415D036A9A0FE96E020E0320EA6E010ED5
:10365000EF24EF6E07D005017B5303E1010E020159
:103660009A27010103010501080E6C25E26F000E87
:103670006D21E36F000E6E21000E6F215C0EE225BE
:10368000E96E030EE321EA6EEFCF74F5090E6C25A7
:10369000E26F000E6D21E36F000E6E21000E6F21B0
:1036A0005C0EE225E96E030EE321EA6EEFCF75F5BD
:1036B0000A0E6C25E26F000E6D21E36F000E6E2185
:1036C000000E6F215C0EE225E96E030EE321EA6E27
:1036D000EFCF76F574516D0804E074514D08D8A40D
:1036E0006CD17551500804E075517008D8A465D1AB
:1036F00076513308D8A461D103015A5306E1010180
:10370000482BD8B4492B57D103015A2D4DD1010173
:103710004A2BD8B44B2B4A514C5DD8A443D14B51C2
:103720004D5DD8A43FD1050E0501E26F00010EECFE
:103730000AF0150E05016C25E26F000E6D21E36F96
:10374000000E6E21000E6F215C0EE225E96E030E65
:10375000E321EA6EEF50E66FEB6BEC6BED6B140E52
:103760006C25EF6F000E6D21F06F000E6E21000EC4
:103770006F215C0EEF25E96E030EF021EA6EEF502B
:10378000F46BF4C503F0026E006A016A0050EB2589
:103790000201896F01500501EC2102018A6F02507C
:1037A0000501ED2102018B6F03500501E6210201A5
:1037B0008C6F1B0E05016C25E26F000E6D21E36F0F
:1037C000000E6E21000E6F215C0EE225E96E030EE5
:1037D000E321EA6EEF50E86BE76BE66FEB6B1A0ED6
:1037E0006C25EF6F000E6D21F06F000E6E21000E44
:1037F0006F215C0EEF25E96E030EF021EA6EEF50AB
:10380000EB25006E000EE621016E000EE721026E30
:10381000000EE821036E00500201892701508A231F
:1038200002508B2303508C23020E895D0501E26F49
:10383000000E02018A590501E36F000E02018B5947
:103840000501E46F000E02018C590501E56FE96F77
:10385000E4C5E8F5E3C5E7F5E2C5E6F5ED6BEC6B2D
:10386000EB6B4BC2EAF50001BAEC0EF003C0E7F2D5
:1038700002C0E6F201C0E5F200C0E4F202017D51AF
:10388000E4277E51E5237F51E6238051E72349A1B8
:1038900006D04B51E45F000EE55BE65BE75B1F0E75
:1038A00005016C25E26F000E6D21E36F000E6E21A5
:1038B000000E6F215C0EE225E96E030EE321EA6E35
:1038C000EF50E66FEB6BEC6BED6B1E0E6C25EF6F44
:1038D000000E6D21F06F000E6E21000E6F215C0E48
:1038E000EF25E96E030EF021EA6EEF50F46BF4C59C
:1038F00003F0026E006A016A0050EB2502018D6F31
:1039000001500501EC2102018E6F02500501ED21ED
:1039100002018F6F03500501E6210201906F1D0E19
:1039200005016C25E26F000E6D21E36F000E6E2124
:10393000000E6F215C0EE225E96E030EE321EA6EB4
:10394000EF50E86BE76BE66FEB6B1C0E6C25EF6FCF
:10395000000E6D21F06F000E6E21000E6F215C0EC7
:10396000EF25E96E030EF021EA6EEF50EB25006EB5
:10397000000EE621016E000EE721026E000EE82126
:10398000036E005002018D2701508E2302508F23B9
:1039900003509023040E0501E26F00010EEC0AF0C3
:1039A00060D3010108D003015A51020805E1010169
:1039B0004A2BD8B44B2B03010501200E6C27000EB7
:1039C0006D236E236F23EBEF17F0010E5C27D8B049
:1039D0005D2BD8B45E2BD8B45F2B1FEF17F002011C
:1039E00075510501775DE26F020176510501785945
:1039F000E36F0201775105017959E46F02017851B3
:103A000005017A59E56FD89002014B350501E22591
:103A1000E66F000EE321E76F000EE421E86F000E71
:103A2000E521E96FF66FE8C5F5F5E7C5F4F5E6C5FC
:103A3000F3F5FA6BF96BF86B4BC2F7F50001F9EC93
:103A40000EF003C06BF502C06AF501C069F500C055
:103A500068F5020149B13AD0D8906431036E633100
:103A6000026E6231016E6131006E03C0E5F502C085
:103A7000E4F501C0E3F5E8CFE2F56BC5F6F56AC5FC
:103A8000F5F569C5F4F568C5F3F503C0FAF502C0AC
:103A9000F9F501C0F8F5E8CFF7F50001F9EC0EF003
:103AA00002015D5105010024606F02015E510501B4
:103AB0000120616F02015F5105010220626F020166
:103AC000605105010320636F40D0020149A13ED03F
:103AD0006431036E6331026E6231016E6131006EDA
:103AE00003320232013200323F0E031603C0E5F505
:103AF00002C0E4F501C0E3F500C0E2F56BC5F6F5E0
:103B00006AC5F5F569C5F4F568C5F3F503C0FAF5BE
:103B100002C0F9F501C0F8F500C0F7F50001F9ECB5
:103B20000EF002015D5105010024606F02015E513B
:103B300005010120616F02015F5105010220626FE2
:103B40000201605105010320636F020149B101D1F7
:103B500063C5E5F562C5E4F561C5E3F560C5E2F569
:103B6000030E0501E76F5C0EE66F000151EC0EF0ED
:103B70000501006A0050685DE66F69516959E76F99
:103B80006A516A59E86F6B516B59E96FD890E63505
:103B90006C6FE7356D6FE8356E6FE9356F6F010E4D
:103BA0006C25E26F000E6D21E36F000E6E21000E9A
:103BB0006F215C0EE225E96E030EE321EA6EEF5001
:103BC000E86BE76BE66FEB6B5C0E6C25E96E030E42
:103BD0006D21EA6EEF50EB25646F000EE621656FF4
:103BE000000EE721666F000EE821676F67530CE156
:103BF00066530AE16551FE08D8B0A9D0FF0A04E176
:103C00006451EF08D8B0A3D0010140A52AD0050126
:103C1000E26BE2510001A6EC03F00501E22B006E1D
:103C200000509EA8FED7AD6E0C0EE25DF2E1080ECC
:103C3000E96E67C5EAF566C5E9F565C5E8F564C5E9
:103C4000E7F500018AEC15F0200E9EA8FED7AD6EB8
:103C50000A0E9EA8FED7AD6E0D0E9EA8FED7AD6EC5
:103C60000101D89002016431036E6331026E62314A
:103C7000016E6131006E03C0E5F502C0E4F501C0DC
:103C8000E3F5E8CFE2F567C5F6F566C5F5F565C578
:103C9000F4F564C5F3F503C0FAF502C0F9F501C007
:103CA000F8F5E8CFF7F50001F9EC0EF002015D51EF
:103CB00005010024606F02015E5105010120616F62
:103CC00002015F5105010220626F0201605105018E
:103CD0000320636F67C56BF566C56AF565C569F551
:103CE00064C568F56BC5E9F56AC5E8F569C5E7F52A
:103CF00068C5E6F5ED6BEC6BEB6B4BC2EAF50001CA
:103D0000BAEC0EF00201755105010024E66F0201C4
:103D1000765105010120E76F02017751050102206C
:103D2000E86F0201785105010320E96FD890020184
:103D30004B350501E65D776F000EE759786F000E91
:103D4000E859796F000EE9597A6FD3EF16F088D1F0
:103D5000020149A186D163C5E5F562C5E4F561C5F7
:103D6000E3F560C5E2F5030E0501E76F5C0EE66F53
:103D7000000151EC0EF005016B31E56F6A31E46F23
:103D80006931E36F6831E26FE533E433E333E23303
:103D9000E533E433E333E233E533E433E333E2336F
:103DA000E533E433E333E233E533E433E333E2335F
:103DB000E533E433E333E233010EE517E235006E19
:103DC000E335016EE435026EE535036E00360136EB
:103DD0000236033600360136023603360036013627
:103DE0000236033600360136023603360036013617
:103DF000023603360036013602360336800E0016D0
:103E00000050685DE66F01506959E76F02506A59CA
:103E1000E86F03506B59E96FE6356C6FE7356D6FEE
:103E2000E8356E6FE9356F6F6C376D376E376F370A
:103E3000FC0E6C17030E6C25E26F000E6D21E36F14
:103E4000000E6E21000E6F215C0EE225E96E030E5E
:103E5000E321EA6EEF50E66FEB6BEC6BED6B020E5D
:103E60006C25EF6F000E6D21F06F000E6E21000EBD
:103E70006F215C0EEF25E96E030EF021EA6EEF5024
:103E8000F46BF36F006A016A0050EB25646F015018
:103E9000EC21656FF351ED21666FF451E621676FF8
:103EA000010E6C25E26F000E6D21E36F000E6E2196
:103EB000000E6F215C0EE225E96E030EE321EA6E2F
:103EC000EF50E86BE76BE66FEB6B5C0E6C25E96E11
:103ED000030E6D21EA6EEF50EB25006E000EE62119
:103EE000016E000EE721026E000EE821036E005005
:103EF0006427015065230250662303506723643D05
:103F000008D0653D06D0663D04D067510F08D8B48F
:103F1000A7D0010140A529D00501E26BE2510001C3
:103F2000A6EC03F00501E22B006E00509EA8FED720
:103F3000AD6E0C0EE25DF2E1080EE96E67C5EAF5C2
:103F400066C5E9F565C5E8F564C5E7F500018AECE5
:103F500015F0200E9EA8FED7AD6E0A0E9EA8FED7C5
:103F6000AD6E0D0E9EA8FED7AD6E02016431036EDC
:103F70006331026E6231016E6131006E03320232D2
:103F8000013200323F0E031603C0E5F502C0E4F52E
:103F900001C0E3F500C0E2F567C5F6F566C5F5F5C5
:103FA00065C5F4F564C5F3F503C0FAF502C0F9F58B
:103FB00001C0F8F500C0F7F50001F9EC0EF00201C0
:103FC0005D5105010024606F02015E510501012071
:103FD000616F02015F5105010220626F02016051B1
:103FE00005010320636F67C56BF566C56AF565C596
:103FF00069F564C568F56BC5E9F56AC5E8F569C595
:10400000E7F568C5E6F5ED6BEC6BEB6B4BC2EAF5DB
:104010000001BAEC0EF00201755105010024E66FB3
:104020000201765105010120E76F02017751050178
:104030000220E86F0201785105010320E96FD89052
:1040400002014B350501E65D776F000EE759786F89
:10405000000EE859796F000EE9597A6FD3EF16F028
:1040600002010001000C5FC30AF05EC309F05DC3EA
:1040700008F05CC307F065EF3AF0016A026A006A73
:10408000036A0301605102E15F5118E0100E616F95
:10409000D8905D375E37003603366051035C02E12D
:1040A0005F51005C07E35F51005ED8A003066051DA
:1040B000035ED88001360236612FEAD7000196EF01
:1040C00020F00AC0E9F509C0E8F508C0E7F507C027
:1040D000E6F5410E0501ED6FC60EEC6F4E0EEB6F6F
:1040E0006D0EEA6F0001BAEC0EF0390E03010024E8
:1040F000076E300E0120086E000E0220096E000EC1
:1041000003200A6E09C000F00AC001F0026A036AC7
:104110000AC05CF309C05BF30AC05EF309C05DF33B
:10412000030E606FE70E5F6F0001A7D700C001F0BC
:1041300003C002F043EF33F00501E26B00010EEC27
:104140000AF0010E0501E26F00010EEC0AF0020E0A
:104150000501E26F00010EEC0AF0030E0501E26FAB
:1041600000010EEC0AF0040E0501E26F00010EECF6
:104170000AF0050E0501E26F00010EEC0AF0000CDA
:104180008188070E03015D6F5D3D01D012D05CC3D5
:1041900000F05D51016E04E0D8900032012EFCD792
:1041A00000A0819600B081868184819481985D070A
:1041B000EBD70001000C03015B6B5A6B5A5303E110
:1041C0005B5108080AE081A2FED75C6B0001D8DFD2
:1041D00003015A2BD8B45B2BF1D7020E6C6F6D6BB9
:1041E000010E6E6F040E6F6F000124EC15F0100EBF
:1041F000006E002EFED7000081B201D0FDD7020E66
:1042000003015C6FC70E5D6F0001EBEC14F003015E
:104210005C2FF8D75C6B0001B3DF03015C6B00011E
:10422000AFDF5BEF33F003019A6B49C3E5F548C399
:10423000E4F547C3E3F546C3E2F5030E0501E76F76
:104240009C0EE66F000151EC0EF003019B6B9B513D
:10425000F90833E39C0E9B25E96E030EEA6ED8B095
:10426000EA2AEF501F0822E209D09C0E9B25E96E36
:10427000030EEA6ED8B0EA2A00A018D0036A9A5159
:104280009825016E995103229C0E03019B25E96E2E
:10429000030EEA6ED8B0EA2AEFCF9EF503C0EAFF1C
:1042A00001C0E9FF9EC5EFFF03019A2B9A51F80860
:1042B00002E2FA0E9B6F9B2BCAD79A51F9080BE3C7
:1042C000036A9A519825E96E99510320EA6E200EEF
:1042D000EF6E9A2BF2D70001ECEF26F0AEC303F09D
:1042E0000301ADC3E9FFAEC3EAFFEF5239E0AEC34D
:1042F000B2F3ADC3B1F3B0C3B4F3AFC3B3F3B4C35C
:1043000003F0B3C3E9FFB4C3EAFFEF5216E0B1C351
:10431000E9FFB2C3EAFFEFCFB5F3B4C303F0B3C311
:10432000E9FFB4C3EAFFEF50B55D07E1B12BD8B4A4
:10433000B22BB32BD8B4B42BE2D7B4C303F0B3C3BE
:10434000E9FFB4C3EAFFEF5205E1ADC301F0AEC32C
:1043500002F009D0AD2BD8B4AE2B0001BFD70301BA
:10436000000E016E026E0001000CAEC3B0F3ADC3CF
:10437000AFF3B0C303F00301AFC3E9FFB0C3EAFF7B
:10438000EF5206E0AF2BD8B4B02B0001F2D70301F7
:10439000AD51AF5D006EAE51B059036E00C001F07B
:1043A000026E0001000C0301AE6B0B0EAD6F020E2E
:1043B000B06FF50EAF6F000191DF01C01CF3030178
:1043C000AE6B0B0EAD6F020EB06FF00EAF6F000153
:1043D00085DF01C01BF30301AE6B0B0EAD6F030E47
:1043E000B06F040EAF6F000179DF01C019F3030154
:1043F000AE6B0B0EAD6F020EB06FFA0EAF6F000119
:104400006DDF01C018F30301AE6B0B0EAD6F020E32
:10441000B06FFF0EAF6F000161DF01C01EF303013B
:10442000AE6B0B0EAD6F030EB06F090EAF6F0001D8
:1044300055DF01C01AF30301AE6B0B0EAD6F030E17
:10444000B06F0E0EAF6F000149DF01C01DF3030115
:10445000AE6B0B0EAD6F030EB06F130EAF6F00019E
:104460003DDF01C01FF30301AE6B0B0EAD6F00010A
:104470007CDF01C028F30301AE6B1CC3ADF3000168
:1044800074DF01C02AF30301AE6B1BC3ADF300015F
:104490006CDF01C029F30301AE6B19C3ADF300015A
:1044A00064DF01C02CF30301AE6B18C3ADF3000150
:1044B0005CDF01C02BF30301AE6B1EC3ADF3000143
:1044C00054DF01C02FF30301AE6B1AC3ADF300013B
:1044D0004CDF01C02DF30301AE6B1DC3ADF3000132
:1044E00044DF01C02EF30301AE6B1FC3ADF3000127
:1044F0003CDF01C030F32AC39CF329C39DF32CC3D6
:104500009EF32BC39FF32FC3A0F32DC3A1F32EC3A0
:10451000A2F330C3A3F30301AE6B1CC3ADF30001E0
:1045200024DF01500301285D246FAE6B1BC3ADF384
:1045300000011BDF01500301285D236FAE6B19C31F
:10454000ADF3000112DF01500301285D216FAE6B56
:1045500018C3ADF3000109DF01500301285D206F8E
:10456000AE6B1EC3ADF3000100DF01500301285DF7
:10457000266FAE6B1AC3ADF30001F7DE01500301E5
:10458000285D226FAE6B1DC3ADF30001EEDE01505E
:104590000301285D256FAE6B1FC3ADF30001E5DE9F
:1045A00001500301285D276F986B996B993D01D0ED
:1045B00022D09A6B9A51070816E3036A9A519C0F0E
:1045C000E96E030E0320EA6E9951EF5C0AE1036A7B
:1045D0009851A50FE96E030E0320EA6E9AC3EFFF10
:1045E000982B9A2BE7D79851080803E1FF0E996F93
:1045F00002D0992BDBD7AE6B1CC3ADF30001B5DE47
:1046000001C02AF3070E03019B6F9B5323E0036A4B
:104610009B51A50FE96E030E0320EA6EEF5218E1DD
:104620009B53D8A49B079BC398F3036A9851A50F8B
:10463000E96E030E0320EA6EEFCFA4F3036AA451E0
:104640009C0FE96E030E0320EA6EEF502A5F02D042
:104650009B07DBD7AE6B1BC3ADF3000186DE01C049
:1046600029F3070E03019B6F9B5323E0036A9B51C1
:10467000A50FE96E030E0320EA6EEF2C18D09B53B2
:10468000D8A49B079BC398F3036A9851A50FE96EC2
:10469000030E0320EA6EEFCFA4F3036AA4519C0F2C
:1046A000E96E030E0320EA6EEF50295F02D09B07EC
:1046B000DBD7040E2A5F295F2A511B0802E21C0E79
:1046C0002A6F29511B0802E21C0E296F0001EEEF30
:1046D00026F0A3C3A8F3A2C3A7F30301A65324E0C3
:1046E000A5C303F0A4C3E9FFA5C3EAFFEF521CE092
:1046F000A8C303F0A751A72BD8B4A82BA96F03C058
:10470000AAF3A5C303F0A451A42BD8B4A52BE96E3A
:1047100003C0EAFFEFCFABF3AAC3EAFFA9C3E9FFE7
:10472000ABC3EFFFA607DAD7A6530CE0A8C303F08C
:10473000A751A72BD8B4A82BE96E03C0EAFFEF6AF4
:10474000A607F2D7A2C301F0A3C302F00001000C38
:1047500003019A6B996B29511B0857E20B0E232515
:104760009B6F9C6BD8B09C2B040E9B259D6F000EFD
:104770009C219E6F010EA36F060EA26F9EC3A5F330
:104780009DC3A4F329C3A6F30001A3DF1B0E0301FD
:10479000986F9851010810E2036A9851060FE96E6C
:1047A000010E0320EA6EEF50200803E0010E295F9E
:1047B00001D002D09807EDD71B0E986F98510108D1
:1047C00010E2036A9851060FE96E010E0320EA6EAB
:1047D000EF50200803E1010E295F01D002D09807B5
:1047E000EDD7010EEA6E060EE96EF2CF9BF3F29E54
:1047F000000E00011EEC04F00A000900F550EE6EF8
:104800000009FBE103019BBFF28E29510E0826E34C
:104810000E0ED8802955006ED89000320050060F39
:104820009C6F010E9D6FD8B09D2B0B0E23259E6FA4
:104830009F6BD8B09F2B040E9E25A06F000E9F216A
:10484000A16F9DC3A3F39CC3A2F3A56FA0C3A4F360
:1048500029C3A6F300013DDF86D0030129511B08BF
:10486000D8A082D00B0E23259B6F9C6BD8B09C2BBD
:10487000040E9B259D6F000E9C219E6F010EA36F61
:10488000060EA26F9EC3A5F39DC3A4F329C3A6F38E
:1048900000011FDF0E0E0301986F9851010810E20E
:1048A000036A9851060FE96E010E0320EA6EEF507D
:1048B000200804E198C39AF3010E986F9807EDD78A
:1048C0009A51295D996F99510E0802E20E0E996F67
:1048D000010EEA6E060EE96EF2CF9BF3F29E000E19
:1048E00000011EEC04F00A000900F550EE6E00090C
:1048F000FBE103019BBFF28E0B0E23259B6F9C6B8C
:10490000D8B09C2B040E9B259D6F000E9C219E6FA2
:10491000010EA36F060EA26F9EC3A5F39DC3A4F361
:104920009AC3A6F30001D5DE0B0E030123259B6F6E
:104930009C6BD8B09C2B040E9B259D6F000E9C2178
:104940009E6F9A519D259F6F000E9E21A06F010EB4
:10495000A36F140EA26FA0C3A5F39FC3A4F399C3C2
:10496000A6F30001B6DE03012351EF0814E2010EA5
:10497000EA6E060EE96EF2CF9BF3F29E000E000186
:104980008FEC04F00A000900F550EE6E0009FBE11F
:1049900003019BBFF28E9A6B996B2A511B08D8B00A
:1049A0006CD00B0E24259B6F9C6BD8B09C2B040EF7
:1049B0009B259D6F000E9C219E6F010EA36F230E01
:1049C000A26F9EC3A5F39DC3A4F32AC3A6F300015F
:1049D00080DE1B0E0301986F9851010810E2036AF4
:1049E0009851230FE96E010E0320EA6EEF50200864
:1049F00003E0010E2A5F01D002D09807EDD71B0E0D
:104A0000986F9851010810E2036A9851230FE96EDC
:104A1000010E0320EA6EEF50200803E1010E2A5F29
:104A200001D002D09807EDD71C0E986F985101085D
:104A300010E2036A9851230FE96E010E0320EA6E1B
:104A4000EF50200804E198C39AF3010E986F98077D
:104A5000EDD7010EEA6E230EE96EF2CF9BF3F29EC4
:104A6000000E00011EEC04F00A000900F550EE6E85
:104A70000009FBE103019BBFF28E2A510E0826E3D9
:104A80000E0ED8802A55006ED89000320050230FA9
:104A90009C6F010E9D6FD8B09D2B0B0E24259E6F31
:104AA0009F6BD8B09F2B040E9E25A06F000E9F21F8
:104AB000A16F9DC3A3F39CC3A2F3A56FA0C3A4F3EE
:104AC0002AC3A6F3000105DE86D003012A511B0884
:104AD000D8A082D00B0E24259B6F9C6BD8B09C2B4A
:104AE000040E9B259D6F000E9C219E6F010EA36FEF
:104AF000230EA26F9EC3A5F39DC3A4F32AC3A6F3FE
:104B00000001E7DD0E0E0301986F9851010810E2D5
:104B1000036A9851230FE96E010E0320EA6EEF50ED
:104B2000200804E198C39AF3010E986F9807EDD717
:104B30009A512A5D996F99510E0802E20E0E996FF3
:104B4000010EEA6E230EE96EF2CF9BF3F29E000E89
:104B500000011EEC04F00A000900F550EE6E000999
:104B6000FBE103019BBFF28E0B0E24259B6F9C6B18
:104B7000D8B09C2B040E9B259D6F000E9C219E6F30
:104B8000010EA36F230EA26F9EC3A5F39DC3A4F3D2
:104B90009AC3A6F300019DDD0B0E030124259B6F34
:104BA0009C6BD8B09C2B040E9B259D6F000E9C2106
:104BB0009E6F9A519D259F6F000E9E21A06F010E42
:104BC000A36F310EA26FA0C3A5F39FC3A4F399C333
:104BD000A6F300017EDD03012451EF0814E2010E6B
:104BE000EA6E230EE96EF2CF9BF3F29E000E0001F7
:104BF0009FEC04F00A000900F550EE6E0009FBE19D
:104C000003019BBFF28E0001EFEF26F00C0E0501B1
:104C1000E66F0001D7EC06F0020EEA6EF00EE96EC8
:104C2000F2CF98F3F29E000EC6EC03F00A000900E2
:104C3000F550EE6E0009FBE1030198BFF28E020E03
:104C4000EA6EF50EE96EF2CF98F3F29E000E0001C7
:104C5000D1EC03F00A000900F550EE6E0009FBE10B
:104C6000030198BFF28E020EEA6EFA0EE96EF2CFE1
:104C700098F3F29E000E0001DCEC03F00A0009003C
:104C8000F550EE6E0009FBE1030198BFF28E020EB3
:104C9000EA6EFF0EE96EF2CF98F3F29E000E00016D
:104CA000E7EC03F00A000900F550EE6E0009FBE1A5
:104CB000030198BFF28E030EEA6E040EE96EF2CF86
:104CC00098F3F29E000E0001F2EC03F00A000900D6
:104CD000F550EE6E0009FBE1030198BFF28E030E62
:104CE000EA6E090EE96EF2CF98F3F29E000E000113
:104CF000FDEC03F00A000900F550EE6E0009FBE13F
:104D0000030198BFF28E030EEA6E0E0EE96EF2CF2B
:104D100098F3F29E000E000108EC04F00A0009006E
:104D2000F550EE6E0009FBE1030198BFF28E030E11
:104D3000EA6E130EE96EF2CF98F3F29E000E0001B8
:104D400013EC04F00A000900F550EE6E0009FBE1D7
:104D5000030198BFF28EEA6A0B0EE96EF2CF98F368
:104D6000F29E000E000172EC03F00A000900F550FB
:104D7000EE6E0009FBE1030198BFF28E010EEA6EB0
:104D8000060EE96EF2CF98F3F29E000E00011EECC3
:104D900004F00A000900F550EE6E0009FBE1030182
:104DA00098BFF28E010EEA6E230EE96EF2CF98F3F1
:104DB000F29E000E00011EEC04F00A000900F550FE
:104DC000EE6E0009FBE1030198BFF28E996B0B0EAA
:104DD000986F000113EF21F0D3EF21F0B9D4030154
:104DE000986B9851000135EC04F00301982B006E8C
:104DF00000509EA8FED7AD6E050E985DF2E1010E43
:104E0000EA6E230EE96E000EEF1008E0EF509EA848
:104E1000FED7AD6EE92AD8B4EA2AF5D7200E9EA8AF
:104E2000FED7AD6E2A0E9EA8FED7AD6E200E9EA8B0
:104E3000FED7AD6E010EEA6E060EE96E000EEF10A3
:104E400008E0EF509EA8FED7AD6EE92AD8B4EA2A52
:104E5000F5D7020E9A6F9A51000143EC04F003015A
:104E60009A2B006E00509EA8FED7AD6E070E9A5D7D
:104E7000F2E1030EA36F7A0EA26F010EA56F230E4F
:104E8000A46F0E0EA66F000124DC0301886B030ED5
:104E9000A36F890EA26F010EA56F310EA46F0E0EC7
:104EA000A66F000116DC0301976B030EA36F5C0E67
:104EB000A26F010EA56F060EA46F0E0EA66F000165
:104EC00008DC03016A6B030EA36F6B0EA26F010E69
:104ED000A56F140EA46F0E0EA66F000169EC23F0EF
:104EE0000301796B0101408F0501E36BE46B000165
:104EF000DEEC06F0030EEA6E7A0EE96E000EEF109D
:104F000010E0EACF99F3E9CF98F3EFCFE6F5D6ECCE
:104F100008F099C3EAFF98C3E9FFE92AD8B4EA2A5E
:104F2000EDD70501E36B010EE46F0001DEEC06F046
:104F3000030EEA6E890EE96E000EEF1010E0EACF64
:104F400099F3E9CF98F3EFCFE6F5D6EC08F099C3E3
:104F5000EAFF98C3E9FFE92AD8B4EA2AEDD70101AC
:104F6000409F0501E36B020EE46F0001DEEC06F0EA
:104F7000030EEA6E5C0EE96E000EEF1010E0EACF51
:104F800099F3E9CF98F3EFCFE6F5D6EC08F099C3A3
:104F9000EAFF98C3E9FFE92AD8B4EA2AEDD7050168
:104FA000E36B030EE46F0001DEEC06F0030EEA6E25
:104FB0006B0EE96E000EEF1010E0EACF99F3E9CF27
:104FC00098F3EFCFE6F5D6EC08F099C3EAFF98C363
:104FD000E9FFE92AD8B4EA2AEDD70301336B346B31
:104FE000000120EF34F00301456B446B436B426BCF
:104FF000E7C2E5F5E6C2E4F5E5C2E3F5E4C2E2F5B1
:10500000030E0501E76F5C0EE66F000151EC0EF038
:1050100003013D6B3C6B3B6B64C33AF3416B406BEC
:105020003F6B65C33EF33A373B373C373D373A3742
:105030003B373C373D373A373B373C373D373A37DC
:105040003B373C373D373A373B373C373D373A37CC
:105050003B373C373D373A373B373C373D37800E9F
:105060003A173DC345F33CC344F33BC343F33AC350
:1050700042F33E5142273F51432340514423415183
:1050800045230A0E4227000E4323442345230501EE
:105090005C6B5C5100017EEC04F005015C2B006E42
:1050A00000509EA8FED7AD6E0A0E5C5DF2E1410E87
:1050B000E96E45C3EAF544C3E9F543C3E8F542C3E5
:1050C000E7F500018AEC15F0200E9EA8FED7AD6E24
:1050D0000A0E9EA8FED7AD6E0D0E9EA8FED7AD6E31
:1050E000C2EF28F003015C6B020E4227000E43233F
:1050F0004423452345530AE1445308E14351010841
:105100000EE2FF0A03E14251000809E25C2B000EA7
:10511000425F020E435B000E445B455BEBD75C5184
:105120000201E42505015D6F000E0201E521050184
:105130005E6F000E0201E62105015F6F000E0201A5
:10514000E7210501606FE56F5FC5E4F55EC5E3F536
:105150005DC5E2F5030EE76F5D0EE66F000151ECF1
:105160000EF00301356B5D0E4225E96E030E4321FF
:10517000EA6EEFCF35F3353B0F0E35170001C3EF65
:1051800028F031D7AFD703015C6B5C5100014FECC5
:1051900004F003015C2B006E00509EA8FED7AD6E9C
:1051A000060E5C5DF2E135C3E3F51B0E0501E46F0D
:1051B0000001F0EC08F0200E9EA8FED7AD6E0A0E9E
:1051C0009EA8FED7AD6E0D0E9EA8FED7AD6E030154
:1051D000596B586B576B566B3551090807E1596B82
:1051E000010E586FF40E576F566B5AD035510A089E
:1051F00007E1596B020E586F710E576F566B50D006
:1052000035510B0807E1596B020E586FEE0E576FC0
:10521000566B46D03551070807E1596B010E586FA0
:10522000770E576F566B3CD035510C0807E1596B20
:10523000030E586F6B0E576F566B32D035510D08F9
:1052400007E1596B030E586FE80E576F566B28D065
:1052500035510E0807E1596B040E586FE20E576F77
:10526000566B1ED0355308E1596B030E586F0D0E67
:10527000576F400E566F14D03551080808E1596B2E
:10528000010E586FB50E576F800E566F09D035510D
:105290000F0806E1596B586B030E576FE80E566FF7
:1052A0005C6B5C5100015DEC04F003015C2B006E53
:1052B00000509EA8FED7AD6E0A0E5C5DF2E1410E75
:1052C000E96E59C3EAF558C3E9F557C3E8F556C383
:1052D000E7F500018AEC15F0200E9EA8FED7AD6E12
:1052E0000A0E9EA8FED7AD6E0D0E9EA8FED7AD6E1F
:1052F00003015931036E5831026E5731016E563138
:10530000006E0332023201320032033202320132C5
:1053100000321F0E031603C05FF302C05EF301C02C
:105320005DF300C05CF34DC3F6F54CC3F5F54BC31C
:10533000F4F54AC3F3F503C0FAF502C0F9F501C06C
:10534000F8F500C0F7F50001F9EC0EF003C055F3D5
:1053500002C054F301C053F300C052F303015C6B6D
:105360005C5100016EEC04F003015C2B006E0050F8
:105370009EA8FED7AD6E0A0E5C5DF2E1410EE96EAD
:1053800055C3EAF554C3E9F553C3E8F552C3E7F54D
:1053900000018AEC15F0200E9EA8FED7AD6E55C315
:1053A000F6F554C3F5F553C3F4F552C3F3F505010F
:1053B000FA6BF96BF86B3C0EF76F0001F9EC0EF02D
:1053C00000C032F3030132513C0DF350525D316F96
:1053D000360E0501E36F040EE46F0001DEEC06F00B
:1053E00032C3E4F5110E0501E56F0001ECEC15F098
:1053F0003A0E0501E66F0001D6EC08F0480E0501F3
:10540000E36F040EE46F0001DEEC06F031C3E4F557
:10541000010E0501E56F0001ECEC15F026EF34F00C
:10542000EACF74F3E9CF73F303016D39F0096F6FBD
:105430006F27E20F706F320F726F6D510F0B702775
:1054400070277227E90F716F712771276C390F0B65
:105450007127722771377237721F72376C510F0BB9
:1054600072276F37070E6E6F0A0E71077227FDE302
:1054700070077127FDE36F077027FDE36E076F2745
:10548000FDE3030EEA6E6E0EE96E070E7315739D53
:10549000E926720EE95CD8B4738DEF50006E08E116
:1054A00073BD06D073B916D073B702D0200E03D0E7
:1054B00073877399300E0026EACF6DF3E9CF6CF352
:1054C00000C0E6F50001D6EC08F06DC3EAFF6CC33E
:1054D000E9FF0301EE5073ADDCD70001000C7E0E36
:1054E0000501E76F0001EFEC06F07E0E0501E76FA6
:1054F0000001EFEC06F00501E76B0001EFEC06F0B0
:105500000501E76B0001EFEC06F07E0E0501E76F89
:105510000001EFEC06F07E0E0501E76F0001EFECF5
:1055200006F00501E76B0001EFEC06F0000C01014D
:105530004099020149B1C0D08CC265F58BC264F5B7
:105540008AC263F589C262F50501716B02015D5182
:10555000050163255E6F02015E51050164215F6FE5
:1055600002015F5105016521606F02016051050173
:105570007121616F61C5E5F560C5E4F55FC5E3F5CF
:105580005EC5E2F5030EE76F5A0EE66F000151ECBF
:105590000EF00501006A0050625D726F635163593D
:1055A000736F64516459746F65516559756FD89004
:1055B00072356A6F73356B6F74356C6F75356D6FDF
:1055C0006DC55DF56CC55CF56BC55BF56AC55AF5D7
:1055D0005D53D8A46ED05C53D8A46BD05B51010846
:1055E000D8A067D003E15A51FE0863E3010E5A25A3
:1055F0006E6F000E5B216F6F000E5C21000E5D214F
:105600005A0E6E25E96E030E6F21EA6EEF50746B31
:10561000736B726F776B5A0E5A25E96E030E5B211E
:10562000EA6EEF507725666F000E7221676F000EED
:105630007321686F000E7421696F69530AE1685322
:1056400008E16751FE0808E2FF0A03E16651EF082E
:1056500003E2000E016EC2D1010E6225006E000E43
:105660006321016E000E6421026E000E6521036E3F
:105670000050665D09E10150675D06E10250685D1A
:1056800003E10350695D06E001014089010E016EEE
:105690000501A4D169C565F568C564F567C563F5FD
:1056A00066C562F5020E5A27000E5B235C235D235C
:1056B0008FD74BD793D1020149A191D18CC265F507
:1056C0008BC264F58AC263F589C262F5010140A507
:1056D0002AD005016E6B6E510001B8EC03F0050194
:1056E0006E2B006E00509EA8FED7AD6E040E6E5D50
:1056F000F2E1410EE96E65C5EAF564C5E9F563C5F9
:10570000E8F562C5E7F500018AEC15F0200E9EA8C9
:10571000FED7AD6E0A0E9EA8FED7AD6E0D0E9EA8EA
:10572000FED7AD6E010105016531716F6431706F97
:1057300063316F6F62316E6F713370336F336E33FD
:10574000713370336F336E33713370336F336E3345
:10575000713370336F336E33713370336F336E3335
:10576000713370336F336E33010E711702015D5167
:1057700005016E255E6F02015E5105016F215F6FAD
:1057800002015F5105017021606F02016051050146
:105790007121616F61C5E5F560C5E4F55FC5E3F5AD
:1057A0005EC5E2F5030EE76F5A0EE66F000151EC9D
:1057B0000EF005016531716F6431706F63316F6F89
:1057C00062316E6F713370336F336E337133703398
:1057D0006F336E33713370336F336E3371337033B5
:1057E0006F336E33713370336F336E3371337033A5
:1057F0006F336E33010E71176E35006E6F35016EAB
:105800007035026E7135036E00360136023603368E
:1058100000360136023603360036013602360336CC
:1058200000360136023603360036013602360336BC
:105830000036013602360336800E00160050625DD7
:10584000726F01506359736F02506459746F035043
:105850006559756F72356A6F73356B6F74356C6F20
:1058600075356D6F6A376B376C376D37FC0E6A179D
:105870006DC55DF56CC55CF56BC55BF56AC55AF524
:105880005D53D8A4AAD05C53D8A4A7D05B5101081B
:10589000D8A0A3D004E15A51FC08D8A09ED0030E92
:1058A0005A256E6F000E5B216F6F000E5C21000E9B
:1058B0005D215A0E6E25E96E030E6F21EA6EEF50E0
:1058C000726F776B786B796B020E5A257B6F000EC7
:1058D0005B217C6F000E5C21000E5D215A0E7B2542
:1058E000E96E030E7C21EA6EEF50806B7F6F006AD9
:1058F000016A00507725666F01507821676F7F51EC
:105900007921686F80517221696F010E5A256E6F7F
:10591000000E5B216F6F000E5C21000E5D215A0EA0
:105920006E25E96E030E6F21EA6EEF50746B736B98
:10593000726F776B5A0E5A25E96E030E5B21EA6E81
:10594000EF507725006E000E7221016E000E73215C
:10595000026E000E7421036E00506627015067230B
:105960000250682303506923663D0AD0673D08D082
:10597000683D06D069510F0803E1000E016E2ED07C
:10598000010E6225006E000E6321016E000E64217F
:10599000026E000E6521036E0050665D09E1015044
:1059A000675D06E10250685D03E10350695D06E052
:1059B00001014089010E016E050110D069C565F530
:1059C00068C564F567C563F566C562F5040E5A27B8
:1059D000000E5B235C235D2353D7A6D60201000192
:1059E000F0EF34F00501E76B0001EFEC06F0FF0E7D
:1059F0000501E76F0001EFEC06F07E0E0501E76F91
:105A00000001EFEC06F03C0E0501E76F0001EFEC42
:105A100006F0180E0501E76F0001EFEC06F0050136
:105A2000E76B0001EFEC06F00501E76B0001EFEC1E
:105A300006F0000C8092FF0E0501F86F000139ECB2
:105A40000AF0500E05015A6F5C6B5B6B5E6B010ECA
:105A50005D6FFF0E5F6F000163EC0AF0015201E021
:105A6000EAD7FF0E0501F86F000139EC0AF0FF0ECE
:105A70000501F86F000139EC0AF0808280926EC354
:105A800076F36FC377F36CC378F36DC379F3510E7C
:105A90000501F06F6FC3F2F56EC3F1F56DC3F4F558
:105AA0006CC3F3F5FF0EF56F00012BEC0EF0FF0E4B
:105AB0000501F86F000139EC0AF001C074F303012D
:105AC000745302E00001F3D7FF0E0501F86F0001E7
:105AD00039EC0AF00150FE0802E00301F5D7FF0E91
:105AE0000501F86F000139EC0AF00301736B726B6A
:105AF000716B01C070F3FF0E0501F86F000139EC06
:105B00000AF0808270C300F071C301F072C302F02A
:105B100073C303F0000C0201499349B11ED0D89021
:105B20009135006E9235016E9335026E9435036E99
:105B300000506D2503015A6F015002016E210301CF
:105B40005B6F025002016F2103015C6F0350020181
:105B5000702103015D6F24D0020149A121D091354C
:105B6000006E9235016E9335026E9435036E0036E9
:105B7000013602360336FC0E001600506D25030177
:105B80005A6F015002016E2103015B6F0250020146
:105B90006F2103015C6F03500201702103015D6FEF
:105BA000010140A919D15DC36FF35CC36EF35BC300
:105BB0006DF35AC36CF300013DDF03C061F302C013
:105BC00060F301C05FF300C05EF3010E03015A25CC
:105BD000626F000E5B21636F000E5C21646F000E2C
:105BE0005D21656F6F6F64C36EF363C36DF362C352
:105BF0006CF300011FDF03C066F302C065F301C050
:105C000064F300C063F302C003F001C002F000C0FF
:105C100001F0006A005003015E250201956F0150FA
:105C200003015F210201966F02500301602102010E
:105C3000976F0350030161210201986F49B138D079
:105C4000976B986B98532FE197532DE19651FF086E
:105C50002AE303E19551EF0826E3D8909535006ECD
:105C60009635016E9735026E9835036E00506D259E
:105C700003015A6F015002016E2103015B6F025054
:105C800002016F2103015C6F0350020170210301C7
:105C90005D6F010E0201E827D8B0E92BD8B4EA2BDA
:105CA000D8B4EB2B04D04983010E016EBDD093D044
:105CB00049A191D0030E03015A255E6F000E5B21AE
:105CC0005F6F000E5C21606F000E5D21616F6F6F72
:105CD00060C36EF35FC36DF35EC36CF30001AADEB5
:105CE00003C062F302C061F301C060F300C05FF360
:105CF00000C067F30301646B656B666B020E5A2587
:105D0000686F000E5B21696F000E5C216A6F000EE8
:105D10005D216B6F6F6F6AC36EF369C36DF368C308
:105D20006CF3000187DE03C06CF302C06BF301C0AB
:105D30006AF300C069F301C003F000C002F0006A1A
:105D4000016A030164510026655101226651022255
:105D500067510322005002019527015096230250FB
:105D6000972303509823953D07D0963D05D0973D46
:105D700003D098510F082BE09535006E9635016ED3
:105D80009735026E9835036E0036013602360336BB
:105D9000FC0E001600506D2503015A6F01500201E0
:105DA0006E2103015B6F025002016F2103015C6FE2
:105DB00003500201702103015D6F010E0201E8270B
:105DC000D8B0E92BD8B4EA2BD8B4EB2B04D0498354
:105DD000010E016E29D0010140B923D0010E02014C
:105DE0009125956F000E9221966F000E9321976F6B
:105DF000000E9421986F010EE827D8B0E92BD8B493
:105E0000EA2BD8B4EB2B8551E85D0AE18651E95DB8
:105E100007E18751EA5D04E18851EB5DD8B449831D
:105E20000101000E016E02010001000C0301626B12
:105E3000636B646B656B81A201D05DD3010140A1EE
:105E4000BED003013353D8B402D00101B8D002014F
:105E5000E851855D006EE9518659016EEA51875916
:105E6000026EEB518859036E0050855D03016C6F23
:105E700001500201865903016D6F025002018759DA
:105E800003016E6F03500201885903016F6FD890B0
:105E9000706B6C35716F6D35726F6E35736FE8CFE7
:105EA000E9F572C3E8F571C3E7F570C3E6F50501DE
:105EB000ED6BEC6BEB6B4BC2EAF50001BAEC0EF04C
:105EC00003C06BF302C06AF301C069F300C068F35A
:105ED00003015931036E5831026E5731016E56314C
:105EE000006E0332023201320032033202320132DA
:105EF00000321F0E031603C06FF302C06EF301C021
:105F00006DF300C06CF36BC3F6F56AC3F5F569C3B6
:105F1000F4F568C3F3F503C0FAF502C0F9F501C062
:105F2000F8F500C0F7F50001F9EC0EF003C055F3E9
:105F300002C054F301C053F300C052F355C3F6F549
:105F400054C3F5F553C3F4F552C3F3F50501FA6BE9
:105F5000F96BF86B3C0EF76F0001F9EC0EF000C026
:105F600032F3030132513C0DF350525D316F360E66
:105F70000501E36F050EE46F0001DEEC06F032C3AD
:105F8000E4F5110E0501E56F0001ECEC15F03A0E99
:105F90000501E66F0001D6EC08F0480E0501E36F3D
:105FA000050EE46F0001DEEC06F031C3E4F5010EEE
:105FB0000501E56F0001ECEC15F073D0010140A183
:105FC00022D003013353D8A402D001011CD0360ED5
:105FD0000501E36F050EE46F0001DEEC06F003013E
:105FE0006C6B6C510001AFEC04F003016C2B006E84
:105FF000E8CFE6F50001D6EC08F0050E03016C5D74
:10600000F0E150D0010140B14CD0030E03016C6FA0
:10601000040E6D6FFF0E6E6F6F6F000124EC15F0B4
:106020000301556B546B02C053F301C052F355C3C7
:10603000F6F554C3F5F553C3F4F552C3F3F5050172
:10604000FA6BF96BF86B3C0EF76F0001F9EC0EF090
:1060500000C032F3030132513C0DF350525D316FF9
:1060600081A201D048D2360E0501E36F050EE46F20
:106070000001DEEC06F032C3E4F5110E0501E56F18
:106080000001ECEC15F03A0E0501E66F0001D6ECCC
:1060900008F031C3E4F5010E0501E56F0001ECECF9
:1060A00015F0030181A201D026D20501E36B050E94
:1060B000E46F0001DEEC06F080B007D0210E050190
:1060C000E66F0001D6EC08F001D08CDC030E030172
:1060D0006C6F050E6D6FFF0E6E6F6F6F000124EC1D
:1060E00015F002C065F301C064F303016451FE0BB7
:1060F000666F65C367F30501E36B040EE46F00018F
:10610000DEEC06F0000EE96E67C36DF366C36CF358
:1061100010EC2AF081A202D00301EDD1030E03019D
:106120006C6F080E6D6FFF0E6E6F6F6F000124ECC9
:1061300015F002C063F301C062F3030163C362F3AD
:10614000636B63336233633362336333623363336A
:1061500062330F0E631781A201D0CDD132510908ED
:1061600009E2210E0501E36F040EE46F0001DEEC8D
:1061700006F008D0240E0501E36F040EE46F000161
:10618000DEEC06F0030162510E0816E1635314E1E0
:10619000330E0501E66F0001D6EC08F0320E050162
:1061A000E66F0001D6EC08F0300E0501E66F000145
:1061B000D6EC08F056D1030162510D0816E1635385
:1061C00014E1320E0501E66F0001D6EC08F0350E41
:1061D0000501E66F0001D6EC08F0360E0501E66F0A
:1061E0000001D6EC08F03DD1030162510C0816E124
:1061F000635314E1320E0501E66F0001D6EC08F09E
:10620000320E0501E66F0001D6EC08F0340E0501F0
:10621000E66F0001D6EC08F024D1030162510B08AF
:1062200016E1635314E1310E0501E66F0001D6EC6F
:1062300008F0390E0501E66F0001D6EC08F0320EC9
:106240000501E66F0001D6EC08F00BD103016251A5
:106250000A0816E1635314E1310E0501E66F0001EF
:10626000D6EC08F0360E0501E66F0001D6EC08F01A
:10627000300E0501E66F0001D6EC08F0F2D0030104
:106280006251090816E1635314E1310E0501E66F0E
:106290000001D6EC08F0320E0501E66F0001D6ECE5
:1062A00008F0380E0501E66F0001D6EC08F0D9D0F1
:1062B00003016251080816E1635314E1310E050130
:1062C000E66F0001D6EC08F0310E0501E66F000123
:1062D000D6EC08F0320E0501E66F0001D6EC08F0AE
:1062E000C0D003016251070816E1635314E1200E88
:1062F0000501E66F0001D6EC08F0390E0501E66FE6
:106300000001D6EC08F0360E0501E66F0001D6EC70
:1063100008F0A7D003016251060816E1635314E1A7
:10632000200E0501E66F0001D6EC08F0380E0501DD
:10633000E66F0001D6EC08F0300E0501E66F0001B3
:10634000D6EC08F08ED003016251050816E16353C4
:1063500014E1200E0501E66F0001D6EC08F0360EC0
:106360000501E66F0001D6EC08F0340E0501E66F7A
:106370000001D6EC08F075D003016251040816E163
:10638000635314E1200E0501E66F0001D6EC08F01E
:10639000350E0501E66F0001D6EC08F0360E05015A
:1063A000E66F0001D6EC08F05CD0030162510308EF
:1063B00016E1635314E1200E0501E66F0001D6ECEF
:1063C00008F0340E0501E66F0001D6EC08F0380E37
:1063D0000501E66F0001D6EC08F043D003016251DD
:1063E000020816E1635314E1200E0501E66F000177
:1063F000D6EC08F0340E0501E66F0001D6EC08F08B
:10640000300E0501E66F0001D6EC08F02AD003013A
:10641000622D15D0635313E1200E0501E66F0001D4
:10642000D6EC08F0330E0501E66F0001D6EC08F05B
:10643000320E0501E66F0001D6EC08F012D0200EF6
:106440000501E66F0001D6EC08F02E0E0501E66F9F
:106450000001D6EC08F0200E0501E66F0001D6EC35
:1064600008F081A202D0030146D00301335327E193
:10647000345308E163C337F362C336F363C339F3BC
:1064800062C338F3342D04D063C337F362C336F3E9
:106490003451020804E163C339F362C338F381A2C3
:1064A00001D029D0342B34510308D8B4346B38517F
:1064B000365D03E13951375D02E0010E336F33532E
:1064C0001AE0360E0501E36F040EE46F0001DEEC06
:1064D00006F003016C6B6C510001BAEC04F003018F
:1064E0006C2B006EE8CFE6F50001D6EC08F0050E47
:1064F00003016C5DF0E10001000C8092FF0E0501CC
:10650000F86F000139EC0AF05CC363F35DC364F318
:106510005BC366F35AC365F3510E0501F06F5DC3AB
:10652000F2F55CC3F1F55BC3F4F55AC3F3F5FF0E66
:10653000F56F00012BEC0EF0FF0E0501F86F000166
:1065400039EC0AF001C061F30301615302E000017C
:10655000F3D7FF0E0501F86F000139EC0AF0015086
:10656000FE0802E00301F5D7020149B330D0030170
:106570005F6B5F5110082AE081B20BD055C151F317
:1065800054C150F353C14FF352C14EF300014EDCDE
:10659000030181B201D0FDD75E6B5E51200814E08B
:1065A00081888088070E606F603D01D00AD080949A
:1065B000808480A6819680B68186818481946007DC
:1065C000F3D781985E2BE9D75F2BD3D7020149A37C
:1065D00043D003015F6B5F5110083EE081B20BD0E6
:1065E00055C151F354C150F353C14FF352C14EF34F
:1065F00000011CDC030181B201D0FDD75E6B5E514E
:10660000200828E081888088070E606F603D01D0F7
:106610001ED0809480840201EC5308E1ED5306E122
:10662000EE5304E1EF5302E181960CD0FF0EEC270C
:10663000D8A0ED27D8A0EE27D8A0EF2780A6819676
:1066400080B681868184819403016007DFD78198B9
:106650005E2BD5D75F2BBFD7FF0E0501F86F00016A
:1066600039EC0AF0FF0E0501F86F000139EC0AF071
:106670008082000E016E78EF37F0010140A716D03E
:10668000000161EF20F002C04DF101C04CF10101A9
:1066900049514D5D06E303E14C51485D02E2F0D7FC
:1066A00005D04C5303E14D5301E1EAD700019CECC6
:1066B00020F0DBEF20F001014091616B606B5F6BBC
:1066C0005E6B409340BB08D0010E03015A6F00017E
:1066D00084EC16F009D0010140AB06D0020E030194
:1066E0005A6F000184EC16F00201995311E1D89021
:1066F0000101566B0201E4350101576F0201E535D6
:106700000101586F0201E6350101596F0BD00201FA
:10671000992D08D0E7C259F1E6C258F1E5C257F108
:10672000E4C256F103015A6B5A51000190EC05F096
:1067300003015A2B006E00509EA8FED7AD6E0C0EC2
:106740005A5DF2E1020EE96E4DC1E3F54CC1E2F58E
:1067500000012FEC16F02F0E9EA8FED7AD6E100E86
:10676000E96E49C1E3F548C1E2F52FEC16F0200EC1
:106770009EA8FED7AD6E010140A54BD003015A6B18
:106780005A510001A3EC05F003015A2B006E005092
:106790009EA8FED7AD6E0A0E5A5DF2E1410EE96E7B
:1067A00059C1EAF558C1E9F557C1E8F556C1E7F511
:1067B00000018AEC15F0200E9EA8FED7AD6E0301F5
:1067C0005A6B5A510001B3EC05F003015A2B006ECD
:1067D00000509EA8FED7AD6E100E5A5DF2E1410E3C
:1067E000E96E90C2EAF58FC2E9F58EC2E8F58DC276
:1067F000E7F500018AEC15F0200E9EA8FED7AD6EDD
:106800000A0E9EA8FED7AD6E0D0E9EA8FED7AD6EE9
:106810000101E7C249F3E6C248F3E5C247F3E4C227
:1068200046F390C24DF38FC24CF38EC24BF38DC230
:106830004AF34DC15BF34CC15AF3000106EF26F059
:106840004DC15BF34CC15AF3C1EF28F00C0E0501AA
:10685000E36F050EE46F0001DEEC06F0020EE96E58
:106860004DC16DF34CC16CF310EC2AF02F0E0501F5
:10687000E66F0001D6EC08F0240E0501E36F050E6B
:10688000E46F0001DEEC06F0100EE96E49C16DF315
:1068900048C16CF310EC2AF0020E03016C6F0B0E72
:1068A0006D6F51C16EF351C16FF3000124EC15F00F
:1068B0000201886B876B866B010E856F05015B6B30
:1068C0004BC25AF5020E5D6F5C6B0001E8EC0EF0F6
:1068D00002C05BF301C05AF30501E96BE86B02C02B
:1068E000E7F501C0E6F588C2EDF587C2ECF586C292
:1068F000EBF585C2EAF50001BAEC0EF00350020197
:10690000905D15E30BE102508F5D11E307E101504B
:106910008E5D0DE303E18D51005C09E2010E8527D8
:10692000D8B0862BD8B4872BD8B4882BC7D7010E04
:10693000855D03015A6F000E0201865903015B6FEA
:10694000000E0201875903015C6F000E0201885995
:1069500003015D6FE8CFE9F55CC3E8F55BC3E7F5DC
:106960005AC3E6F50501ED6BEC6BEB6B4BC2EAF538
:106970000001BAEC0EF003C05EF302C05DF301C08B
:106980005CF300C05BF3D890006A03015B35016ED5
:106990005C35026E5D35036E005002018D5DEC6F5B
:1069A00001508E59ED6F02508F59EE6F0350905980
:1069B000EF6FEB6BEA6BE96BE86B8CC294F28BC206
:1069C00093F28AC292F289C291F20501E36B050E3D
:1069D000E46F0001DEEC06F06FEC2AF097EF2AF08E
:1069E000010140A510D003015A6B5A510001C7ECB8
:1069F00005F003015A2B006E00509EA8FED7AD6E25
:106A0000110E5A5DF2E10501E36B050EE46F000122
:106A1000DEEC06F0F2EC2CF00201EB51885DD8A020
:106A200080D20EE1EA51875DD8A07BD209E1E9511D
:106A3000865DD8A076D204E1E851855DD8A071D2F8
:106A400000018BEC2DF0020E0201915D03015A6FE3
:106A5000000E0201925903015B6F000E020193596F
:106A600003015C6F000E0201945903015D6FE8CFD2
:106A7000E9F55CC3E8F55BC3E7F55AC3E6F5050144
:106A8000ED6BEC6BEB6B4BC2EAF50001BAEC0EF070
:106A900003C065F102C064F101C063F100C062F19E
:106AA00002017D510101622702017E510101632330
:106AB00002017F510101642302018051010165231C
:106AC000020149A108D04B510101625F000E635BD6
:106AD000645B655B0201995316E1D89001015A6B22
:106AE00062355B6F63355C6F64355D6F020E4F6FAF
:106AF0004E6B74C269F173C268F172C267F171C200
:106B000066F114D00201992D12D065C15DF164C106
:106B10005CF163C15BF162C15AF101014F6B010E7F
:106B20004E6F696B686B676B4BC266F102018092B6
:106B3000FF0E0501F86F000139EC0AF0500E050157
:106B40005A6F5C6B5B6B020E5E6F5D6BFF0E5F6F6F
:106B5000000163EC0AF0015202E00201E9D7FF0EE6
:106B60000501F86F000139EC0AF0FF0E0501F86F1E
:106B7000000139EC0AF080825DC155F15CC154F12D
:106B80005BC153F15AC152F1010166515A25006EA1
:106B900067515B21016E68515C21026E69515D2174
:106BA000036E0050525D0AE10150535D07E102504F
:106BB000545D04E10350555DD8B4A3D184A00FD037
:106BC0004C2BD8B44D2B49514D5D07E303E14C519B
:106BD000485D03E24D6B010E4C6F50D552D080AA38
:106BE0000DD04C51D8B44D074C2F06D04D5304E175
:106BF00049C14DF148C14CF141D543D084A420D0C6
:106C0000515110081DE20501E36B050EE46F000110
:106C1000DEEC06F02B0E0501E66F0001D6EC08F065
:106C200001015107020E03016C6F0B0E6D6F51C114
:106C30006EF351C16FF3000124EC15F021D0010176
:106C400084A21FD0513D01D01CD00501E36B050E7D
:106C5000E46F0001DEEC06F02D0E0501E66F000189
:106C6000D6EC08F00101512B020E03016C6F0B0EE4
:106C70006D6F51C16EF351C16FF3000124EC15F03B
:106C80000101616B606B5F6B5E6B83AE41D0010E87
:106C90005E27D8B05F2BD8B4602BD8B4612B010E1F
:106CA00003015A6F0001B0EC06F0010140B32FD090
:106CB000615307E1605305E15F5303E15E51F90859
:106CC00026E20501E36B050EE46F0001DEEC06F041
:106CD0003E0E0501E66F0001D6EC08F0010140818F
:106CE0004093020149B312D000018BEC2DF0020158
:106CF00049B30CD098C294F297C293F296C292F222
:106D000095C291F2000116EC2FF002010101BDD7EE
:106D100040B324D05E5306E15F5304E1605302E1C7
:106D200061531CE061531AE1605318E15F5316E1AF
:106D30005E51F90813E340830501E36B050EE46F30
:106D40000001DEEC06F06FEC2AF0140E03015A6F1E
:106D50000001B0EC06F0010194D7BFD040A31AD0D7
:106D60005E5306E15F5304E1605302E1615312E0B8
:106D700040930501E36B050EE46F0001DEEC06F0C5
:106D8000F2EC2CF0140E03015A6F0001B0EC06F087
:106D9000A5D0010140A3A1D040AD2AD0506B000185
:106DA0009CEC20F00501E36B050EE46F0001DEECC6
:106DB00006F00101408F03015A6B5A510001D8ECD3
:106DC00005F003015A2B006EE8CFE6F50001D6EC82
:106DD00008F00E0E03015A5DF0E10101409F030E21
:106DE00003015A6F000184EC16F00101408B409DB5
:106DF00084A22CD0408B4751455DD8A0452B030180
:106E00005A6B5A510001E8EC05F003015A2B006E51
:106E100000509EA8FED7AD6E130E5A5DF2E145C13B
:106E2000E3F51B0E0501E46F0001F0EC08F0200E05
:106E30009EA8FED7AD6E0A0E9EA8FED7AD6E0D0EB3
:106E40009EA8FED7AD6E0101408D2DD084A42BD01D
:106E5000408B45510008D8A0450703015A6B5A5191
:106E60000001E8EC05F003015A2B006E00509EA8CB
:106E7000FED7AD6E130E5A5DF2E145C1E3F51B0E70
:106E80000501E46F0001F0EC08F0200E9EA8FED78B
:106E9000AD6E0A0E9EA8FED7AD6E0D0E9EA8FED753
:106EA000AD6E0101408D83AE11D040AB0FD0020E0C
:106EB00003016C6F0B0E6D6FFF0E6E6F6F6F000135
:106EC00024EC15F03DEF33F009D0010183AE04D07E
:106ED00040BB02D0D6D601D05FD7000155C15DF3CB
:106EE00054C15CF353C15BF352C15AF37DEF32F0EE
:106EF00001014E5152274F515323000E5423552365
:106F000044D6020149B309D098C294F297C293F2D1
:106F100096C292F295C291F203D049A301D001D05A
:106F20007CD50001EEEF3AF0F86AD09EFE0E006EBE
:106F3000060E016E020EE96E000EEA6EEE6A002E7B
:106F4000FDD7012EFBD7EA6AE96A0A0EAF6EA60EDC
:106F5000AC6E900EAB6EC180C182C184C196056AD1
:106F6000066A1E0E01016A6F210E6B6F610E6C6F57
:106F7000210E6D6F120E6E6F3C0E6F6F410E706FB3
:106F8000400E716F210E726F7C0E736F380E746F2E
:106F9000540E756F560E766F550E776F180E786F0C
:106FA000200E796F550E7A6F7B6F7C6F780E7D6F38
:106FB000200E7E6F550E7F6F540E806F550E816FC1
:106FC000780E826F200E836F550E846F560E856F7C
:106FD000540E866F780E876F200E886F540E896F5F
:106FE000550E8A6F540E8B6F780E8C6F1C0E8D6F42
:106FF000220E8E6F620E8F6F220E906F100E916FA9
:10700000380E926F550E936F946F956F180E966FA2
:10701000380E976F550E986F540E996F550E9A6FE4
:10702000180E9B6F380E9C6F540E9D6F550E9E6F01
:10703000560E9F6F180EA06FA16B450EA26F7C0EAF
:10704000A36F410EA46FA56BA66B450EA76F7D0EB7
:10705000A86F410EA96FAA6BAB6B450EAC6F7E0E8D
:10706000AD6F400EAE6FAF6B780EB06F150EB16F97
:10707000140EB26F150EB36F780EB46FB56F140E99
:10708000B66F150EB76F140EB86F780EB96F7C0E11
:10709000BA6F540EBB6F560EBC6F550EBD6F440ECB
:1070A000BE6F240EBF6F540EC06F780EC16F540EAA
:1070B000C26F480EC36F7E0EC46F090EC56F7E0E81
:1070C000C66F490EC76FC86F380EC96F450ECA6FBD
:1070D000CB6FCC6F380ECD6FCE6F450ECF6F440E99
:1070E000D06F450ED16F380ED26FD36F450ED46F6F
:1070F000460ED56F440ED66F380ED76F3C0ED86F44
:10710000410ED96FDA6F210EDB6F7C0EDC6F3C0E07
:10711000DD6F410EDE6F420EDF6F200EE06F7C0EE2
:10712000E16F0C0EE26F510EE36F500EE46F510EE3
:10713000E56F3C0EE66F380EE76F450EE86F440EC4
:10714000E96F450EEA6F380EEB6F3C0EEC6F410EA7
:10715000ED6F400EEE6F410EEF6F3C0EF06FF16B76
:10716000F26BF36BF46BF56B200EF66F480EF76F56
:107170003E0EF86F490EF96F620EFA6FFB6BFC6BF7
:10718000FD6BFE6BFF6B0201006B016B026B036B0F
:10719000046B400E056F680E066F3E0E076F090EFA
:1071A000086F020E096F200E0A6F540E0B6F560EF9
:1071B0000C6F550E0D6F780E0E6F0F6B440E106F27
:1071C0007E0E116F410E126F136B380E146F440E4A
:1071D000156F460E166F450E176F380E186F3C0E62
:1071E000196F400E1A6F420E1B6F210E1C6F7C0E22
:1071F0001D6F1E6F090E1F6F050E206F216F780E19
:10720000226F7C0E236F090E246F110E256F210E45
:10721000266F7C0E276F7E0E286F250E296F2A6F32
:10722000260E2B6F180E2C6FC290C180C182C184B4
:10723000C196290E926E8082020E936E900E946E0D
:10724000C00E956E96809682968403015A6B5A51B1
:107250000001C5EC04F003015A2B006E00509EA8FB
:10726000FED7AD6E260E5A5DF2E10001FDEF05F08E
:1072700087EF06F011EC07F02FEF09F00501E36B43
:10728000E46B0001DEEC06F00101408F03015A6B54
:107290005A510001E1EC04F003015A2B006EE8CFD3
:1072A000E6F50001D6EC08F00E0E03015A5DF0E1A0
:1072B0000101409F090E0501E36F010EE46F00011B
:1072C000DEEC06F003015A6B5A510001F1EC04F0B8
:1072D00003015A2B006EE8CFE6F50001D6EC08F06A
:1072E0000B0E03015A5DF0E10501E36B020EE46F42
:1072F0000001DEEC06F003015A6B5A510001FFEC6D
:1073000004F003015A2B006EE8CFE6F50001D6EC3D
:1073100008F00E0E03015A5DF0E1030E0501E26F65
:1073200000010EEC0AF00501E36B030EE46F0001AF
:10733000DEEC06F0010140A515D0408F03015A6B29
:107340005A5100010FEC05F003015A2B006EE8CFF3
:10735000E6F50001D6EC08F0050E03015A5DF0E1F8
:107360000101409F2A0E0501E36F030EE46F000147
:10737000DEEC06F0010140A715D0408F03015A6BE7
:107380005A5100011AEC05F003015A2B006EE8CFA8
:10739000E6F50001D6EC08F0070E03015A5DF0E1B6
:1073A0000101409F040E0501E26F00010EEC0AF09E
:1073B000050E0501E26F00010EEC0AF036EF0BF04E
:1073C000010140A510D003015A6B5A51000126EC6F
:1073D00005F003015A2B006E00509EA8FED7AD6E3B
:1073E000130E5A5DF2E1000139EF0FF0010140A5E3
:1073F00010D003015A6B5A51000138EC05F003011B
:107400005A2B006E00509EA8FED7AD6E180E5A5D26
:10741000F2E1000150EF15F0010140A511D0030188
:107420005A6B5A5100014DEC05F003015A2B006EC6
:1074300000509EA8FED7AD6E0F0E5A5DF2E101011D
:10744000496B486B4D6B010E4C6F436B456B476B43
:1074500003015A6B000184EC16F0010140A526D00F
:1074600003015A6B5A5100015DEC05F003015A2BE0
:10747000006E00509EA8FED7AD6E0D0E5A5DF2E173
:10748000100EE96E49C1E3F548C1E2F500012FECA9
:1074900016F0200E9EA8FED7AD6E0A0E9EA8FED74F
:1074A000AD6E0D0E9EA8FED7AD6E0101D650D7CFA2
:1074B00003F003015A6FD7CF5BF35F6B5E6BD7CFDF
:1074C0005DF35C6F000133EF20F0010140A551D066
:1074D000200E9EA8FED7AD6E0A0E9EA8FED7AD6EFA
:1074E0000D0E9EA8FED7AD6E446B4451415D41E345
:1074F00003015A6B5A5100016FEC05F003015A2B3E
:10750000006E00509EA8FED7AD6E0B0E5A5DF2E1E4
:1075100044C1E3F51B0E0501E46F0001F0EC08F037
:107520003D0E9EA8FED7AD6E200E9EA8FED7AD6E76
:10753000036A010144519A0FE96E020E0320EA6EBC
:10754000EFCF5AF35AC3E3F51B0E0501E46F0001B8
:10755000F0EC08F0200E9EA8FED7AD6E0A0E9EA895
:10756000FED7AD6E0D0E9EA8FED7AD6E0101442B69
:10757000BCD703015A6B5A5100017FEC05F003019F
:107580005A2B006E00509EA8FED7AD6E0B0E5A5DB2
:10759000F2E147C1E3F51B0E0501E46F0001F0ECD9
:1075A00008F0200E9EA8FED7AD6E0A0E9EA8FED74C
:1075B000AD6E0D0E9EA8FED7AD6E280E0101516F67
:1075C000020E03016C6F0B0E6D6F51C16EF351C152
:1075D0006FF3000124EC15F03DEF33F001014C2B6B
:1075E000D8B44D2B49514D5D07E303E14C51485D43
:0E75F00003E24D6B010E4C6F0001EED703005D
:020000040030CA
:0E00000000220C0E000180000FC00FE00F4028
:00000001FF
